Archive member included because of file (symbol)

f:/microsemi/softconsole_v4.0/arm-none-eabi-gcc/bin/../lib/gcc/arm-none-eabi/4.9.3/../../../../arm-none-eabi/lib/armv7-m\libg_nano.a(lib_a-errno.o)
                              ./MotorControl_Drivers/firmware/CMSIS/startup_gcc/newlib_stubs.o (__errno)
f:/microsemi/softconsole_v4.0/arm-none-eabi-gcc/bin/../lib/gcc/arm-none-eabi/4.9.3/../../../../arm-none-eabi/lib/armv7-m\libg_nano.a(lib_a-exit.o)
                              f:/microsemi/softconsole_v4.0/arm-none-eabi-gcc/bin/../lib/gcc/arm-none-eabi/4.9.3/../../../../arm-none-eabi/lib/armv7-m/crt0.o (exit)
f:/microsemi/softconsole_v4.0/arm-none-eabi-gcc/bin/../lib/gcc/arm-none-eabi/4.9.3/../../../../arm-none-eabi/lib/armv7-m\libg_nano.a(lib_a-impure.o)
                              f:/microsemi/softconsole_v4.0/arm-none-eabi-gcc/bin/../lib/gcc/arm-none-eabi/4.9.3/../../../../arm-none-eabi/lib/armv7-m\libg_nano.a(lib_a-exit.o) (_global_impure_ptr)
f:/microsemi/softconsole_v4.0/arm-none-eabi-gcc/bin/../lib/gcc/arm-none-eabi/4.9.3/../../../../arm-none-eabi/lib/armv7-m\libg_nano.a(lib_a-init.o)
                              f:/microsemi/softconsole_v4.0/arm-none-eabi-gcc/bin/../lib/gcc/arm-none-eabi/4.9.3/../../../../arm-none-eabi/lib/armv7-m/crt0.o (__libc_init_array)
f:/microsemi/softconsole_v4.0/arm-none-eabi-gcc/bin/../lib/gcc/arm-none-eabi/4.9.3/../../../../arm-none-eabi/lib/armv7-m\libg_nano.a(lib_a-memcpy.o)
                              ./MotorControl_Drivers/firmware/drivers/mss_sys_services/mss_sys_services.o (memcpy)
f:/microsemi/softconsole_v4.0/arm-none-eabi-gcc/bin/../lib/gcc/arm-none-eabi/4.9.3/../../../../arm-none-eabi/lib/armv7-m\libg_nano.a(lib_a-memset.o)
                              f:/microsemi/softconsole_v4.0/arm-none-eabi-gcc/bin/../lib/gcc/arm-none-eabi/4.9.3/../../../../arm-none-eabi/lib/armv7-m/crt0.o (memset)

Allocating common symbols
Common symbol       size              file

g_usbd_msc_media_ops
                    0x4               ./MotorControl_Drivers/firmware/drivers/mss_usb/mss_usb_device_msd.o
g_hall_sensor_pol   0x1               ./MotorControl_App/MCCalc.o
g_LX_PWM_freq_kHz   0x4               ./MotorControl_App/MCCalc.o
g_usbd_msc_user_speed
                    0x1               ./MotorControl_Drivers/firmware/drivers/mss_usb/mss_usb_device_msd.o
g_bot_cbw           0x20              ./MotorControl_Drivers/firmware/drivers/mss_usb/mss_usb_device_msd.o
g_theta_factor      0x4               ./MotorControl_App/MCCalc.o
g_pwm_period_st     0x4               ./MotorControl_App/MCCalc.o
g_en_angle_cnt_max  0x4               ./MotorControl_App/MCCalc.o
speedbuf            0x4               ./MotorControl_App/MCFPGAIF.o
g_mss_usbd_printer_ops
                    0x4               ./MotorControl_Drivers/firmware/drivers/mss_usb/mss_usb_device_printer.o
g_usbd_hid_user_speed
                    0x1               ./MotorControl_Drivers/firmware/drivers/mss_usb/mss_usb_device_hid.o
g_slew_count_st     0x4               ./MotorControl_App/MCCalc.o
g_en_speed_window   0x4               ./MotorControl_App/MCCalc.o
g_speed_scale       0x4               ./MotorControl_App/MCCalc.o
g_bot_state         0x1               ./MotorControl_Drivers/firmware/drivers/mss_usb/mss_usb_device_msd.o
g_encoder_steps     0x4               ./MotorControl_App/USBMsgHandler.o
gd_tx_ep            0x14              ./MotorControl_Drivers/firmware/drivers/mss_usb/mss_usb_device_cif.o
g_pwm_period        0x4               ./MotorControl_App/MCCalc.o
g_base_addr         0x4               ./MotorControl_App/MCFPGAIF.o
g_slew_count        0x4               ./MotorControl_App/MCCalc.o
g_rate_count        0x4               ./MotorControl_App/MCCalc.o
g_en_speed_factor   0x4               ./MotorControl_App/MCCalc.o
cep_state           0x1               ./MotorControl_Drivers/firmware/drivers/mss_usb/mss_usb_device_cif.o
g_usbd_cdc_user_speed
                    0x1               ./MotorControl_Drivers/firmware/drivers/mss_usb/mss_usb_device_cdc.o
g_rate_count_st     0x4               ./MotorControl_App/MCCalc.o
g_bldc1             0x18              ./MotorControl_App/MCCalc.o
currentbuf          0x4               ./MotorControl_App/MCFPGAIF.o
g_pwm_gain          0x4               ./MotorControl_App/MCCalc.o
g_adc_scale_st      0x4               ./MotorControl_App/MCCalc.o
g_sense_response    0x12              ./MotorControl_Drivers/firmware/drivers/mss_usb/mss_usb_device_msd.o
g_algorithm         0x1               ./MotorControl_App/MCCalc.o
g_stepper           0x38              ./MotorControl_App/MCCalc.o
usbd_cdc_vcp_ops    0x4               ./MotorControl_Drivers/firmware/drivers/mss_usb/mss_usb_device_cdc.o
g_usbd_vendor_user_speed
                    0x1               ./MotorControl_Drivers/firmware/drivers/mss_usb/mss_usb_device_vendor.o
gd_rx_ep            0x14              ./MotorControl_Drivers/firmware/drivers/mss_usb/mss_usb_device_cif.o
g_usbd_class_cb     0x4               ./MotorControl_Drivers/firmware/drivers/mss_usb/mss_usb_device.o
g_usbd_user_descr_cb
                    0x4               ./MotorControl_Drivers/firmware/drivers/mss_usb/mss_usb_device.o
g_adc_scale         0x4               ./MotorControl_App/MCCalc.o
g_mc_bldc_foc       0x4c              ./MotorControl_App/MCCalc.o
g_speed_descale     0x4               ./MotorControl_App/MCCalc.o
g_en_angle_factor   0x4               ./MotorControl_App/MCCalc.o

Discarded input sections

 .text          0x00000000        0x0 f:/microsemi/softconsole_v4.0/arm-none-eabi-gcc/bin/../lib/gcc/arm-none-eabi/4.9.3/armv7-m/crti.o
 .data          0x00000000        0x0 f:/microsemi/softconsole_v4.0/arm-none-eabi-gcc/bin/../lib/gcc/arm-none-eabi/4.9.3/armv7-m/crti.o
 .bss           0x00000000        0x0 f:/microsemi/softconsole_v4.0/arm-none-eabi-gcc/bin/../lib/gcc/arm-none-eabi/4.9.3/armv7-m/crti.o
 .data          0x00000000        0x4 f:/microsemi/softconsole_v4.0/arm-none-eabi-gcc/bin/../lib/gcc/arm-none-eabi/4.9.3/armv7-m/crtbegin.o
 .text          0x00000000       0x74 f:/microsemi/softconsole_v4.0/arm-none-eabi-gcc/bin/../lib/gcc/arm-none-eabi/4.9.3/../../../../arm-none-eabi/lib/armv7-m/crt0.o
 .data          0x00000000        0x0 f:/microsemi/softconsole_v4.0/arm-none-eabi-gcc/bin/../lib/gcc/arm-none-eabi/4.9.3/../../../../arm-none-eabi/lib/armv7-m/crt0.o
 .bss           0x00000000        0x0 f:/microsemi/softconsole_v4.0/arm-none-eabi-gcc/bin/../lib/gcc/arm-none-eabi/4.9.3/../../../../arm-none-eabi/lib/armv7-m/crt0.o
 .ARM.extab     0x00000000        0x0 f:/microsemi/softconsole_v4.0/arm-none-eabi-gcc/bin/../lib/gcc/arm-none-eabi/4.9.3/../../../../arm-none-eabi/lib/armv7-m/crt0.o
 .ARM.exidx     0x00000000        0x8 f:/microsemi/softconsole_v4.0/arm-none-eabi-gcc/bin/../lib/gcc/arm-none-eabi/4.9.3/../../../../arm-none-eabi/lib/armv7-m/crt0.o
 .text          0x00000000        0xe ./MotorControl_Drivers/firmware/hal/CortexM3/GNU/hal.o
 .data          0x00000000        0x0 ./MotorControl_Drivers/firmware/hal/CortexM3/GNU/hal.o
 .bss           0x00000000        0x0 ./MotorControl_Drivers/firmware/hal/CortexM3/GNU/hal.o
 .data          0x00000000        0x0 ./MotorControl_Drivers/firmware/hal/CortexM3/GNU/hw_reg_access.o
 .bss           0x00000000        0x0 ./MotorControl_Drivers/firmware/hal/CortexM3/GNU/hw_reg_access.o
 .text          0x00000000        0x0 ./MotorControl_Drivers/firmware/hal/CortexM3/cortex_nvic.o
 .data          0x00000000        0x0 ./MotorControl_Drivers/firmware/hal/CortexM3/cortex_nvic.o
 .bss           0x00000000        0x0 ./MotorControl_Drivers/firmware/hal/CortexM3/cortex_nvic.o
 .text.NVIC_init
                0x00000000        0x4 ./MotorControl_Drivers/firmware/hal/CortexM3/cortex_nvic.o
 .text.NVIC_set_handler
                0x00000000        0x4 ./MotorControl_Drivers/firmware/hal/CortexM3/cortex_nvic.o
 .text.NVIC_set_priority
                0x00000000        0x4 ./MotorControl_Drivers/firmware/hal/CortexM3/cortex_nvic.o
 .text.NVIC_enable_interrupt
                0x00000000        0x4 ./MotorControl_Drivers/firmware/hal/CortexM3/cortex_nvic.o
 .text.NVIC_disable_interrupt
                0x00000000        0x4 ./MotorControl_Drivers/firmware/hal/CortexM3/cortex_nvic.o
 .text.NVIC_clear_interrupt
                0x00000000        0x4 ./MotorControl_Drivers/firmware/hal/CortexM3/cortex_nvic.o
 .text          0x00000000        0x0 ./MotorControl_Drivers/firmware/drivers_config/sys_config/sys_config.o
 .data          0x00000000        0x0 ./MotorControl_Drivers/firmware/drivers_config/sys_config/sys_config.o
 .bss           0x00000000        0x0 ./MotorControl_Drivers/firmware/drivers_config/sys_config/sys_config.o
 .text          0x00000000        0x0 ./MotorControl_Drivers/firmware/drivers/mss_usb/mss_usb_common_cif.o
 .data          0x00000000        0x0 ./MotorControl_Drivers/firmware/drivers/mss_usb/mss_usb_common_cif.o
 .bss           0x00000000        0x0 ./MotorControl_Drivers/firmware/drivers/mss_usb/mss_usb_common_cif.o
 .text          0x00000000        0x0 ./MotorControl_Drivers/firmware/drivers/mss_usb/mss_usb_device.o
 .data          0x00000000        0x0 ./MotorControl_Drivers/firmware/drivers/mss_usb/mss_usb_device.o
 .bss           0x00000000        0x0 ./MotorControl_Drivers/firmware/drivers/mss_usb/mss_usb_device.o
 .text.MSS_USBD_tx_ep_stall
                0x00000000       0x2c ./MotorControl_Drivers/firmware/drivers/mss_usb/mss_usb_device.o
 .text.MSS_USBD_tx_ep_clr_stall
                0x00000000       0x2a ./MotorControl_Drivers/firmware/drivers/mss_usb/mss_usb_device.o
 .text.MSS_USBD_rx_ep_stall
                0x00000000       0x2c ./MotorControl_Drivers/firmware/drivers/mss_usb/mss_usb_device.o
 .text.MSS_USBD_rx_ep_clr_stall
                0x00000000       0x2a ./MotorControl_Drivers/firmware/drivers/mss_usb/mss_usb_device.o
 .text.MSS_USBD_cep_flush_fifo
                0x00000000       0x14 ./MotorControl_Drivers/firmware/drivers/mss_usb/mss_usb_device.o
 .text.MSS_USBD_get_hwcore_info
                0x00000000        0x4 ./MotorControl_Drivers/firmware/drivers/mss_usb/mss_usb_device.o
 .text.MSS_USBD_set_dev_address
                0x00000000        0xc ./MotorControl_Drivers/firmware/drivers/mss_usb/mss_usb_device.o
 .text.MSS_USBD_get_dev_address
                0x00000000        0xc ./MotorControl_Drivers/firmware/drivers/mss_usb/mss_usb_device.o
 .text.MSS_USBD_dev_force_resume
                0x00000000       0x10 ./MotorControl_Drivers/firmware/drivers/mss_usb/mss_usb_device.o
 .text.MSS_USBD_set_isoupdate
                0x00000000       0x10 ./MotorControl_Drivers/firmware/drivers/mss_usb/mss_usb_device.o
 .text.MSS_USBD_tx_ep_clr_isoupdate
                0x00000000       0x10 ./MotorControl_Drivers/firmware/drivers/mss_usb/mss_usb_device.o
 .text.MSS_USBD_tx_ep_is_fifo_notempty
                0x00000000       0x10 ./MotorControl_Drivers/firmware/drivers/mss_usb/mss_usb_device.o
 .text.MSS_USBD_rx_ep_is_fifo_full
                0x00000000       0x10 ./MotorControl_Drivers/firmware/drivers/mss_usb/mss_usb_device.o
 .text.MSS_USBD_enable_usbirq
                0x00000000       0x10 ./MotorControl_Drivers/firmware/drivers/mss_usb/mss_usb_device.o
 .text.MSS_USBD_disable_usbirq
                0x00000000       0x10 ./MotorControl_Drivers/firmware/drivers/mss_usb/mss_usb_device.o
 .text.MSS_USBD_tx_ep_disable_irq
                0x00000000       0x18 ./MotorControl_Drivers/firmware/drivers/mss_usb/mss_usb_device.o
 .text.MSS_USBD_rx_ep_disable_irq
                0x00000000       0x18 ./MotorControl_Drivers/firmware/drivers/mss_usb/mss_usb_device.o
 .text.MSS_USBD_tx_ep_enable_irq
                0x00000000       0x14 ./MotorControl_Drivers/firmware/drivers/mss_usb/mss_usb_device.o
 .text.MSS_USBD_rx_ep_enable_irq
                0x00000000       0x14 ./MotorControl_Drivers/firmware/drivers/mss_usb/mss_usb_device.o
 .text.MSS_USBD_cep_enable_irq
                0x00000000       0x14 ./MotorControl_Drivers/firmware/drivers/mss_usb/mss_usb_device.o
 .text.MSS_USBD_cep_disable_irq
                0x00000000       0x14 ./MotorControl_Drivers/firmware/drivers/mss_usb/mss_usb_device.o
 .text          0x00000000        0x0 ./MotorControl_Drivers/firmware/drivers/mss_usb/mss_usb_device_cdc.o
 .data          0x00000000        0x0 ./MotorControl_Drivers/firmware/drivers/mss_usb/mss_usb_device_cdc.o
 .bss           0x00000000        0x0 ./MotorControl_Drivers/firmware/drivers/mss_usb/mss_usb_device_cdc.o
 .text.CDC_get_descriptor_cb
                0x00000000       0x1c ./MotorControl_Drivers/firmware/drivers/mss_usb/mss_usb_device_cdc.o
 .text.CDC_deinit_cb
                0x00000000       0x10 ./MotorControl_Drivers/firmware/drivers/mss_usb/mss_usb_device_cdc.o
 .text.CDC_process_request_cb
                0x00000000       0x18 ./MotorControl_Drivers/firmware/drivers/mss_usb/mss_usb_device_cdc.o
 .text.CDC_cep_datain_cb
                0x00000000       0x14 ./MotorControl_Drivers/firmware/drivers/mss_usb/mss_usb_device_cdc.o
 .text.CDC_cep_dataout_cb
                0x00000000       0x14 ./MotorControl_Drivers/firmware/drivers/mss_usb/mss_usb_device_cdc.o
 .text.CDC_init_cb
                0x00000000       0x84 ./MotorControl_Drivers/firmware/drivers/mss_usb/mss_usb_device_cdc.o
 .text.CDC_dataout_cb
                0x00000000       0x20 ./MotorControl_Drivers/firmware/drivers/mss_usb/mss_usb_device_cdc.o
 .text.CDC_datain_cb
                0x00000000       0x40 ./MotorControl_Drivers/firmware/drivers/mss_usb/mss_usb_device_cdc.o
 .text.MSS_USBD_CDC_init
                0x00000000       0x1c ./MotorControl_Drivers/firmware/drivers/mss_usb/mss_usb_device_cdc.o
 .text.MSS_USBD_CDC_tx
                0x00000000       0x1c ./MotorControl_Drivers/firmware/drivers/mss_usb/mss_usb_device_cdc.o
 .text.MSS_USBD_CDC_rx_prepare
                0x00000000       0x1c ./MotorControl_Drivers/firmware/drivers/mss_usb/mss_usb_device_cdc.o
 .text.MSS_USBD_CDC_get_state
                0x00000000        0xc ./MotorControl_Drivers/firmware/drivers/mss_usb/mss_usb_device_cdc.o
 .data.usbd_cdc_class_cb
                0x00000000       0x20 ./MotorControl_Drivers/firmware/drivers/mss_usb/mss_usb_device_cdc.o
 .bss.g_usbd_cdc_state
                0x00000000        0x1 ./MotorControl_Drivers/firmware/drivers/mss_usb/mss_usb_device_cdc.o
 .data.cdc_conf_descr
                0x00000000       0x4b ./MotorControl_Drivers/firmware/drivers/mss_usb/mss_usb_device_cdc.o
 COMMON         0x00000000        0x8 ./MotorControl_Drivers/firmware/drivers/mss_usb/mss_usb_device_cdc.o
 .text          0x00000000        0x0 ./MotorControl_Drivers/firmware/drivers/mss_usb/mss_usb_device_cif.o
 .data          0x00000000        0x0 ./MotorControl_Drivers/firmware/drivers/mss_usb/mss_usb_device_cif.o
 .bss           0x00000000        0x0 ./MotorControl_Drivers/firmware/drivers/mss_usb/mss_usb_device_cif.o
 .text.MSS_USBD_CIF_get_hwcore_info
                0x00000000       0x60 ./MotorControl_Drivers/firmware/drivers/mss_usb/mss_usb_device_cif.o
 .text          0x00000000        0x0 ./MotorControl_Drivers/firmware/drivers/mss_usb/mss_usb_device_hid.o
 .data          0x00000000        0x0 ./MotorControl_Drivers/firmware/drivers/mss_usb/mss_usb_device_hid.o
 .bss           0x00000000        0x0 ./MotorControl_Drivers/firmware/drivers/mss_usb/mss_usb_device_hid.o
 .text.MSS_USBD_HID_rx_done
                0x00000000        0xc ./MotorControl_Drivers/firmware/drivers/mss_usb/mss_usb_device_hid.o
 .text          0x00000000        0x0 ./MotorControl_Drivers/firmware/drivers/mss_usb/mss_usb_device_msd.o
 .data          0x00000000        0x0 ./MotorControl_Drivers/firmware/drivers/mss_usb/mss_usb_device_msd.o
 .bss           0x00000000        0x0 ./MotorControl_Drivers/firmware/drivers/mss_usb/mss_usb_device_msd.o
 .text.USBD_MSC_get_descriptor_cb
                0x00000000       0x74 ./MotorControl_Drivers/firmware/drivers/mss_usb/mss_usb_device_msd.o
 .text.USBD_MSC_deinit_cb
                0x00000000       0x10 ./MotorControl_Drivers/firmware/drivers/mss_usb/mss_usb_device_msd.o
 .text.USBD_MSC_init_cb
                0x00000000       0xfc ./MotorControl_Drivers/firmware/drivers/mss_usb/mss_usb_device_msd.o
 .text.USBD_MSC_process_request_cb
                0x00000000       0xd8 ./MotorControl_Drivers/firmware/drivers/mss_usb/mss_usb_device_msd.o
 .text.MSS_USBD_MSC_init
                0x00000000       0x1c ./MotorControl_Drivers/firmware/drivers/mss_usb/mss_usb_device_msd.o
 .text.MSS_USBD_MSC_get_state
                0x00000000        0xc ./MotorControl_Drivers/firmware/drivers/mss_usb/mss_usb_device_msd.o
 .text.USBD_MSC_prepare_sense_data
                0x00000000        0xc ./MotorControl_Drivers/firmware/drivers/mss_usb/mss_usb_device_msd.o
 .text.USBD_MSC_abort_cbw
                0x00000000       0x12 ./MotorControl_Drivers/firmware/drivers/mss_usb/mss_usb_device_msd.o
 .text.USBD_MSC_send_data
                0x00000000       0x28 ./MotorControl_Drivers/firmware/drivers/mss_usb/mss_usb_device_msd.o
 .text.USBD_MSC_receive_data
                0x00000000       0x18 ./MotorControl_Drivers/firmware/drivers/mss_usb/mss_usb_device_msd.o
 .text.USBD_MSC_send_csw
                0x00000000       0x1c ./MotorControl_Drivers/firmware/drivers/mss_usb/mss_usb_device_msd.o
 .text.USBD_MSC_process_read_10
                0x00000000       0x90 ./MotorControl_Drivers/firmware/drivers/mss_usb/mss_usb_device_msd.o
 .text.USBD_MSC_process_write_10
                0x00000000       0x8c ./MotorControl_Drivers/firmware/drivers/mss_usb/mss_usb_device_msd.o
 .text.USBD_MSC_process_cbw
                0x00000000      0x1b8 ./MotorControl_Drivers/firmware/drivers/mss_usb/mss_usb_device_msd.o
 .text.USBD_MSC_BOT_fsm
                0x00000000      0x2f8 ./MotorControl_Drivers/firmware/drivers/mss_usb/mss_usb_device_msd.o
 .text.USBD_MSC_data_in_cb
                0x00000000       0x24 ./MotorControl_Drivers/firmware/drivers/mss_usb/mss_usb_device_msd.o
 .text.USBD_MSC_data_out_cb
                0x00000000       0x24 ./MotorControl_Drivers/firmware/drivers/mss_usb/mss_usb_device_msd.o
 .bss.g_tx_buf_ptr
                0x00000000        0x4 ./MotorControl_Drivers/firmware/drivers/mss_usb/mss_usb_device_msd.o
 .data.mode_sense_response
                0x00000000        0xc ./MotorControl_Drivers/firmware/drivers/mss_usb/mss_usb_device_msd.o
 .bss.g_rx_current_lba_addr
                0x00000000        0x4 ./MotorControl_Drivers/firmware/drivers/mss_usb/mss_usb_device_msd.o
 .bss.g_rx_buf_len
                0x00000000        0x4 ./MotorControl_Drivers/firmware/drivers/mss_usb/mss_usb_device_msd.o
 .bss.g_botin_events
                0x00000000        0x1 ./MotorControl_Drivers/firmware/drivers/mss_usb/mss_usb_device_msd.o
 .data.g_current_command_csw
                0x00000000       0x10 ./MotorControl_Drivers/firmware/drivers/mss_usb/mss_usb_device_msd.o
 .data.msc_hs_conf_descr
                0x00000000       0x20 ./MotorControl_Drivers/firmware/drivers/mss_usb/mss_usb_device_msd.o
 .bss.lun_capacity
                0x00000000       0x30 ./MotorControl_Drivers/firmware/drivers/mss_usb/mss_usb_device_msd.o
 .bss.g_botout_events
                0x00000000        0x1 ./MotorControl_Drivers/firmware/drivers/mss_usb/mss_usb_device_msd.o
 .bss.get_max_lun_response
                0x00000000        0x1 ./MotorControl_Drivers/firmware/drivers/mss_usb/mss_usb_device_msd.o
 .bss.format_capacity_list
                0x00000000        0xc ./MotorControl_Drivers/firmware/drivers/mss_usb/mss_usb_device_msd.o
 .data.usb_msd_class_cb
                0x00000000       0x20 ./MotorControl_Drivers/firmware/drivers/mss_usb/mss_usb_device_msd.o
 .data.msc_fs_conf_descr
                0x00000000       0x20 ./MotorControl_Drivers/firmware/drivers/mss_usb/mss_usb_device_msd.o
 .bss.g_tx_current_lba_addr
                0x00000000        0x4 ./MotorControl_Drivers/firmware/drivers/mss_usb/mss_usb_device_msd.o
 .bss.g_tx_buf_len
                0x00000000        0x4 ./MotorControl_Drivers/firmware/drivers/mss_usb/mss_usb_device_msd.o
 .rodata.str1.1
                0x00000000        0x2 ./MotorControl_Drivers/firmware/drivers/mss_usb/mss_usb_device_msd.o
 .bss.g_usbd_msc_state
                0x00000000        0x1 ./MotorControl_Drivers/firmware/drivers/mss_usb/mss_usb_device_msd.o
 .bss.g_rx_buf_ptr
                0x00000000        0x4 ./MotorControl_Drivers/firmware/drivers/mss_usb/mss_usb_device_msd.o
 COMMON         0x00000000       0x3b ./MotorControl_Drivers/firmware/drivers/mss_usb/mss_usb_device_msd.o
 .text          0x00000000        0x0 ./MotorControl_Drivers/firmware/drivers/mss_usb/mss_usb_device_printer.o
 .data          0x00000000        0x0 ./MotorControl_Drivers/firmware/drivers/mss_usb/mss_usb_device_printer.o
 .bss           0x00000000        0x0 ./MotorControl_Drivers/firmware/drivers/mss_usb/mss_usb_device_printer.o
 .text.USBD_printer_deinit
                0x00000000       0x20 ./MotorControl_Drivers/firmware/drivers/mss_usb/mss_usb_device_printer.o
 .text.USBD_printer_get_descriptor
                0x00000000       0x1c ./MotorControl_Drivers/firmware/drivers/mss_usb/mss_usb_device_printer.o
 .text.USBD_printer_process_request
                0x00000000       0x14 ./MotorControl_Drivers/firmware/drivers/mss_usb/mss_usb_device_printer.o
 .text.USBD_printer_data_in
                0x00000000       0x28 ./MotorControl_Drivers/firmware/drivers/mss_usb/mss_usb_device_printer.o
 .text.USBD_printer_data_out
                0x00000000       0x28 ./MotorControl_Drivers/firmware/drivers/mss_usb/mss_usb_device_printer.o
 .text.USBD_printer_cep_datain
                0x00000000       0x14 ./MotorControl_Drivers/firmware/drivers/mss_usb/mss_usb_device_printer.o
 .text.USBD_printer_cep_dataout
                0x00000000       0x14 ./MotorControl_Drivers/firmware/drivers/mss_usb/mss_usb_device_printer.o
 .text.USBD_printer_init
                0x00000000       0x88 ./MotorControl_Drivers/firmware/drivers/mss_usb/mss_usb_device_printer.o
 .text.MSS_USBD_printer_init
                0x00000000        0xc ./MotorControl_Drivers/firmware/drivers/mss_usb/mss_usb_device_printer.o
 .text.MSS_USBD_PRINTER_set_cb_handler
                0x00000000        0xc ./MotorControl_Drivers/firmware/drivers/mss_usb/mss_usb_device_printer.o
 .text.MSS_USBD_PRINTER_write
                0x00000000        0xc ./MotorControl_Drivers/firmware/drivers/mss_usb/mss_usb_device_printer.o
 .text.MSS_USBD_PRINTER_read_prepare
                0x00000000        0xc ./MotorControl_Drivers/firmware/drivers/mss_usb/mss_usb_device_printer.o
 .text.MSS_USBD_printer_get_state
                0x00000000        0xc ./MotorControl_Drivers/firmware/drivers/mss_usb/mss_usb_device_printer.o
 .data.fs_conf_descr
                0x00000000       0x20 ./MotorControl_Drivers/firmware/drivers/mss_usb/mss_usb_device_printer.o
 .data.conf_descr
                0x00000000       0x20 ./MotorControl_Drivers/firmware/drivers/mss_usb/mss_usb_device_printer.o
 .bss.g_printer_events
                0x00000000        0x1 ./MotorControl_Drivers/firmware/drivers/mss_usb/mss_usb_device_printer.o
 .data.usb_printer_class_cb
                0x00000000       0x20 ./MotorControl_Drivers/firmware/drivers/mss_usb/mss_usb_device_printer.o
 .bss.g_usbd_printer_state
                0x00000000        0x1 ./MotorControl_Drivers/firmware/drivers/mss_usb/mss_usb_device_printer.o
 COMMON         0x00000000        0x4 ./MotorControl_Drivers/firmware/drivers/mss_usb/mss_usb_device_printer.o
 .text          0x00000000        0x0 ./MotorControl_Drivers/firmware/drivers/mss_usb/mss_usb_device_vendor.o
 .data          0x00000000        0x0 ./MotorControl_Drivers/firmware/drivers/mss_usb/mss_usb_device_vendor.o
 .bss           0x00000000        0x0 ./MotorControl_Drivers/firmware/drivers/mss_usb/mss_usb_device_vendor.o
 .text.USBD_VENDOR_get_descriptor_cb
                0x00000000       0x74 ./MotorControl_Drivers/firmware/drivers/mss_usb/mss_usb_device_vendor.o
 .text.USBD_VENDOR_process_request_cb
                0x00000000       0x20 ./MotorControl_Drivers/firmware/drivers/mss_usb/mss_usb_device_vendor.o
 .text.USBD_VENDOR_cep_data_in_cb
                0x00000000        0x4 ./MotorControl_Drivers/firmware/drivers/mss_usb/mss_usb_device_vendor.o
 .text.USBD_VENDOR_cep_data_out_cb
                0x00000000        0x4 ./MotorControl_Drivers/firmware/drivers/mss_usb/mss_usb_device_vendor.o
 .text.USBD_VENDOR_init_cb
                0x00000000       0xc0 ./MotorControl_Drivers/firmware/drivers/mss_usb/mss_usb_device_vendor.o
 .text.USBD_VENDOR_data_in_cb
                0x00000000       0x30 ./MotorControl_Drivers/firmware/drivers/mss_usb/mss_usb_device_vendor.o
 .text.USBD_VENDOR_data_out_cb
                0x00000000       0x30 ./MotorControl_Drivers/firmware/drivers/mss_usb/mss_usb_device_vendor.o
 .text.MSS_USBD_VENDOR_init
                0x00000000       0x14 ./MotorControl_Drivers/firmware/drivers/mss_usb/mss_usb_device_vendor.o
 .text.USBD_VENDOR_deinit_cb
                0x00000000        0x4 ./MotorControl_Drivers/firmware/drivers/mss_usb/mss_usb_device_vendor.o
 .bss.g_req_rx_data
                0x00000000       0x19 ./MotorControl_Drivers/firmware/drivers/mss_usb/mss_usb_device_vendor.o
 .data.usb_vendor_class_cb
                0x00000000       0x20 ./MotorControl_Drivers/firmware/drivers/mss_usb/mss_usb_device_vendor.o
 .data.g_bulk_tx_data
                0x00000000       0x40 ./MotorControl_Drivers/firmware/drivers/mss_usb/mss_usb_device_vendor.o
 .bss.g_intr_rx_data
                0x00000000       0x40 ./MotorControl_Drivers/firmware/drivers/mss_usb/mss_usb_device_vendor.o
 .data.g_req_tx_data
                0x00000000       0x19 ./MotorControl_Drivers/firmware/drivers/mss_usb/mss_usb_device_vendor.o
 .data.vendor_hs_conf_descr
                0x00000000       0x2e ./MotorControl_Drivers/firmware/drivers/mss_usb/mss_usb_device_vendor.o
 .bss.g_bulk_rx_data
                0x00000000       0x40 ./MotorControl_Drivers/firmware/drivers/mss_usb/mss_usb_device_vendor.o
 .data.g_intr_tx_data
                0x00000000       0x40 ./MotorControl_Drivers/firmware/drivers/mss_usb/mss_usb_device_vendor.o
 .data.vendor_fs_conf_descr
                0x00000000       0x2e ./MotorControl_Drivers/firmware/drivers/mss_usb/mss_usb_device_vendor.o
 COMMON         0x00000000        0x1 ./MotorControl_Drivers/firmware/drivers/mss_usb/mss_usb_device_vendor.o
 .text          0x00000000        0x0 ./MotorControl_Drivers/firmware/drivers/mss_usb/mss_usb_host.o
 .data          0x00000000        0x0 ./MotorControl_Drivers/firmware/drivers/mss_usb/mss_usb_host.o
 .bss           0x00000000        0x0 ./MotorControl_Drivers/firmware/drivers/mss_usb/mss_usb_host.o
 .text          0x00000000        0x0 ./MotorControl_Drivers/firmware/drivers/mss_usb/mss_usb_host_cif.o
 .data          0x00000000        0x0 ./MotorControl_Drivers/firmware/drivers/mss_usb/mss_usb_host_cif.o
 .bss           0x00000000        0x0 ./MotorControl_Drivers/firmware/drivers/mss_usb/mss_usb_host_cif.o
 .text          0x00000000        0x0 ./MotorControl_Drivers/firmware/drivers/mss_usb/mss_usb_host_msc.o
 .data          0x00000000        0x0 ./MotorControl_Drivers/firmware/drivers/mss_usb/mss_usb_host_msc.o
 .bss           0x00000000        0x0 ./MotorControl_Drivers/firmware/drivers/mss_usb/mss_usb_host_msc.o
 .text          0x00000000        0x0 ./MotorControl_Drivers/firmware/drivers/mss_sys_services/mss_comblk.o
 .data          0x00000000        0x0 ./MotorControl_Drivers/firmware/drivers/mss_sys_services/mss_comblk.o
 .bss           0x00000000        0x0 ./MotorControl_Drivers/firmware/drivers/mss_sys_services/mss_comblk.o
 .text.send_cmd_opcode
                0x00000000       0x1c ./MotorControl_Drivers/firmware/drivers/mss_sys_services/mss_comblk.o
 .text.MSS_COMBLK_init
                0x00000000       0xa4 ./MotorControl_Drivers/firmware/drivers/mss_sys_services/mss_comblk.o
 .text.MSS_COMBLK_send_cmd_with_ptr
                0x00000000       0xcc ./MotorControl_Drivers/firmware/drivers/mss_sys_services/mss_comblk.o
 .text.MSS_COMBLK_send_cmd
                0x00000000      0x104 ./MotorControl_Drivers/firmware/drivers/mss_sys_services/mss_comblk.o
 .text.MSS_COMBLK_send_paged_cmd
                0x00000000       0xf0 ./MotorControl_Drivers/firmware/drivers/mss_sys_services/mss_comblk.o
 .text          0x00000000        0x0 ./MotorControl_Drivers/firmware/drivers/mss_sys_services/mss_sys_services.o
 .data          0x00000000        0x0 ./MotorControl_Drivers/firmware/drivers/mss_sys_services/mss_sys_services.o
 .bss           0x00000000        0x0 ./MotorControl_Drivers/firmware/drivers/mss_sys_services/mss_sys_services.o
 .text.asynchronous_event_handler
                0x00000000       0xa8 ./MotorControl_Drivers/firmware/drivers/mss_sys_services/mss_sys_services.o
 .text.isp_page_read_handler
                0x00000000       0x64 ./MotorControl_Drivers/firmware/drivers/mss_sys_services/mss_sys_services.o
 .text.isp_sys_completion_handler
                0x00000000       0x2c ./MotorControl_Drivers/firmware/drivers/mss_sys_services/mss_sys_services.o
 .text.request_completion_handler
                0x00000000       0x14 ./MotorControl_Drivers/firmware/drivers/mss_sys_services/mss_sys_services.o
 .text.signal_request_start
                0x00000000       0x20 ./MotorControl_Drivers/firmware/drivers/mss_sys_services/mss_sys_services.o
 .text.wait_for_request_completion
                0x00000000       0x18 ./MotorControl_Drivers/firmware/drivers/mss_sys_services/mss_sys_services.o
 .text.write_ptr_value_into_array
                0x00000000       0x12 ./MotorControl_Drivers/firmware/drivers/mss_sys_services/mss_sys_services.o
 .text.execute_service
                0x00000000       0x3c ./MotorControl_Drivers/firmware/drivers/mss_sys_services/mss_sys_services.o
 .text.MSS_SYS_init
                0x00000000       0x3c ./MotorControl_Drivers/firmware/drivers/mss_sys_services/mss_sys_services.o
 .text.MSS_SYS_get_serial_number
                0x00000000       0x14 ./MotorControl_Drivers/firmware/drivers/mss_sys_services/mss_sys_services.o
 .text.MSS_SYS_get_user_code
                0x00000000       0x14 ./MotorControl_Drivers/firmware/drivers/mss_sys_services/mss_sys_services.o
 .text.MSS_SYS_get_design_version
                0x00000000       0x14 ./MotorControl_Drivers/firmware/drivers/mss_sys_services/mss_sys_services.o
 .text.MSS_SYS_get_device_certificate
                0x00000000       0x14 ./MotorControl_Drivers/firmware/drivers/mss_sys_services/mss_sys_services.o
 .text.MSS_SYS_get_secondary_device_certificate
                0x00000000       0x5c ./MotorControl_Drivers/firmware/drivers/mss_sys_services/mss_sys_services.o
 .text.MSS_SYS_flash_freeze
                0x00000000       0x84 ./MotorControl_Drivers/firmware/drivers/mss_sys_services/mss_sys_services.o
 .text.MSS_SYS_128bit_aes
                0x00000000       0x6c ./MotorControl_Drivers/firmware/drivers/mss_sys_services/mss_sys_services.o
 .text.MSS_SYS_256bit_aes
                0x00000000       0x6c ./MotorControl_Drivers/firmware/drivers/mss_sys_services/mss_sys_services.o
 .text.MSS_SYS_sha256
                0x00000000       0x40 ./MotorControl_Drivers/firmware/drivers/mss_sys_services/mss_sys_services.o
 .text.MSS_SYS_hmac
                0x00000000       0x5c ./MotorControl_Drivers/firmware/drivers/mss_sys_services/mss_sys_services.o
 .text.MSS_SYS_key_tree
                0x00000000       0x66 ./MotorControl_Drivers/firmware/drivers/mss_sys_services/mss_sys_services.o
 .text.MSS_SYS_challenge_response
                0x00000000       0x44 ./MotorControl_Drivers/firmware/drivers/mss_sys_services/mss_sys_services.o
 .text.MSS_SYS_nrbg_reset
                0x00000000       0x54 ./MotorControl_Drivers/firmware/drivers/mss_sys_services/mss_sys_services.o
 .text.MSS_SYS_nrbg_self_test
                0x00000000       0x48 ./MotorControl_Drivers/firmware/drivers/mss_sys_services/mss_sys_services.o
 .text.MSS_SYS_nrbg_instantiate
                0x00000000       0x38 ./MotorControl_Drivers/firmware/drivers/mss_sys_services/mss_sys_services.o
 .text.MSS_SYS_nrbg_generate
                0x00000000       0x44 ./MotorControl_Drivers/firmware/drivers/mss_sys_services/mss_sys_services.o
 .text.MSS_SYS_nrbg_reseed
                0x00000000       0x28 ./MotorControl_Drivers/firmware/drivers/mss_sys_services/mss_sys_services.o
 .text.MSS_SYS_nrbg_uninstantiate
                0x00000000       0x4c ./MotorControl_Drivers/firmware/drivers/mss_sys_services/mss_sys_services.o
 .text.MSS_SYS_zeroize_device
                0x00000000       0x64 ./MotorControl_Drivers/firmware/drivers/mss_sys_services/mss_sys_services.o
 .text.MSS_SYS_check_digest
                0x00000000       0x90 ./MotorControl_Drivers/firmware/drivers/mss_sys_services/mss_sys_services.o
 .text.MSS_SYS_start_isp
                0x00000000       0xac ./MotorControl_Drivers/firmware/drivers/mss_sys_services/mss_sys_services.o
 .text.MSS_SYS_initiate_iap
                0x00000000       0xdc ./MotorControl_Drivers/firmware/drivers/mss_sys_services/mss_sys_services.o
 .text.MSS_SYS_puf_create_activation_code
                0x00000000       0x60 ./MotorControl_Drivers/firmware/drivers/mss_sys_services/mss_sys_services.o
 .text.MSS_SYS_puf_delete_activation_code
                0x00000000       0x60 ./MotorControl_Drivers/firmware/drivers/mss_sys_services/mss_sys_services.o
 .text.MSS_SYS_puf_get_number_of_keys
                0x00000000       0x74 ./MotorControl_Drivers/firmware/drivers/mss_sys_services/mss_sys_services.o
 .text.MSS_SYS_puf_enroll_key
                0x00000000       0x88 ./MotorControl_Drivers/firmware/drivers/mss_sys_services/mss_sys_services.o
 .text.MSS_SYS_puf_delete_key
                0x00000000       0x64 ./MotorControl_Drivers/firmware/drivers/mss_sys_services/mss_sys_services.o
 .text.MSS_SYS_puf_fetch_key
                0x00000000       0x68 ./MotorControl_Drivers/firmware/drivers/mss_sys_services/mss_sys_services.o
 .text.MSS_SYS_puf_export_keycodes
                0x00000000       0x6c ./MotorControl_Drivers/firmware/drivers/mss_sys_services/mss_sys_services.o
 .text.MSS_SYS_puf_import_keycodes
                0x00000000       0x6c ./MotorControl_Drivers/firmware/drivers/mss_sys_services/mss_sys_services.o
 .text.MSS_SYS_puf_fetch_ecc_public_key
                0x00000000       0x64 ./MotorControl_Drivers/firmware/drivers/mss_sys_services/mss_sys_services.o
 .text.MSS_SYS_puf_get_random_seed
                0x00000000       0x64 ./MotorControl_Drivers/firmware/drivers/mss_sys_services/mss_sys_services.o
 .text.MSS_SYS_ecc_point_multiplication
                0x00000000       0x7c ./MotorControl_Drivers/firmware/drivers/mss_sys_services/mss_sys_services.o
 .text.MSS_SYS_ecc_point_addition
                0x00000000       0x7c ./MotorControl_Drivers/firmware/drivers/mss_sys_services/mss_sys_services.o
 .text.MSS_SYS_ecc_get_base_point
                0x00000000       0x24 ./MotorControl_Drivers/firmware/drivers/mss_sys_services/mss_sys_services.o
 .text.MSS_SYS_start_clock_monitor
                0x00000000       0x90 ./MotorControl_Drivers/firmware/drivers/mss_sys_services/mss_sys_services.o
 .text.MSS_SYS_stop_clock_monitor
                0x00000000       0x90 ./MotorControl_Drivers/firmware/drivers/mss_sys_services/mss_sys_services.o
 .text.MSS_SYS_enable_puf_power_down
                0x00000000       0x90 ./MotorControl_Drivers/firmware/drivers/mss_sys_services/mss_sys_services.o
 .text.MSS_SYS_disable_puf_power_down
                0x00000000       0x90 ./MotorControl_Drivers/firmware/drivers/mss_sys_services/mss_sys_services.o
 .text.MSS_SYS_clear_lock_parity
                0x00000000       0x90 ./MotorControl_Drivers/firmware/drivers/mss_sys_services/mss_sys_services.o
 .text.MSS_SYS_clear_mesh_short
                0x00000000       0x90 ./MotorControl_Drivers/firmware/drivers/mss_sys_services/mss_sys_services.o
 .rodata        0x00000000       0x60 ./MotorControl_Drivers/firmware/drivers/mss_sys_services/mss_sys_services.o
 .bss.g_event_handler
                0x00000000        0x4 ./MotorControl_Drivers/firmware/drivers/mss_sys_services/mss_sys_services.o
 .bss.g_request_in_progress
                0x00000000        0x1 ./MotorControl_Drivers/firmware/drivers/mss_sys_services/mss_sys_services.o
 .bss.g_isp_completion_handler
                0x00000000        0x4 ./MotorControl_Drivers/firmware/drivers/mss_sys_services/mss_sys_services.o
 .bss.g_isp_page_read_handler
                0x00000000        0x4 ./MotorControl_Drivers/firmware/drivers/mss_sys_services/mss_sys_services.o
 .bss.g_response
                0x00000000        0x2 ./MotorControl_Drivers/firmware/drivers/mss_sys_services/mss_sys_services.o
 .bss.g_mode    0x00000000        0x1 ./MotorControl_Drivers/firmware/drivers/mss_sys_services/mss_sys_services.o
 .data.g_initial_envm_cr
                0x00000000        0x4 ./MotorControl_Drivers/firmware/drivers/mss_sys_services/mss_sys_services.o
 .bss.g_last_response_length
                0x00000000        0x2 ./MotorControl_Drivers/firmware/drivers/mss_sys_services/mss_sys_services.o
 .data.wait_for_clock_switch
                0x00000000        0x1 ./MotorControl_Drivers/firmware/drivers/mss_sys_services/mss_sys_services.o
 .bss.g_isp_response
                0x00000000        0x2 ./MotorControl_Drivers/firmware/drivers/mss_sys_services/mss_sys_services.o
 .bss.g_initial_mssddr_facc1_cr
                0x00000000        0x4 ./MotorControl_Drivers/firmware/drivers/mss_sys_services/mss_sys_services.o
 .bss.g_initial_mssddr_facc2_cr
                0x00000000        0x4 ./MotorControl_Drivers/firmware/drivers/mss_sys_services/mss_sys_services.o
 .text          0x00000000        0x0 ./MotorControl_Drivers/firmware/drivers/mss_nvm/mss_nvm.o
 .data          0x00000000        0x0 ./MotorControl_Drivers/firmware/drivers/mss_nvm/mss_nvm.o
 .bss           0x00000000        0x0 ./MotorControl_Drivers/firmware/drivers/mss_nvm/mss_nvm.o
 .text.request_nvm_access
                0x00000000       0x4c ./MotorControl_Drivers/firmware/drivers/mss_nvm/mss_nvm.o
 .text.release_ctrl_access
                0x00000000       0x40 ./MotorControl_Drivers/firmware/drivers/mss_nvm/mss_nvm.o
 .text.wait_nvm_ready
                0x00000000       0x2c ./MotorControl_Drivers/firmware/drivers/mss_nvm/mss_nvm.o
 .text.get_ctrl_access
                0x00000000       0x44 ./MotorControl_Drivers/firmware/drivers/mss_nvm/mss_nvm.o
 .text.NVM_write
                0x00000000      0x214 ./MotorControl_Drivers/firmware/drivers/mss_nvm/mss_nvm.o
 .text.NVM_unlock
                0x00000000      0x120 ./MotorControl_Drivers/firmware/drivers/mss_nvm/mss_nvm.o
 .rodata.g_nvm  0x00000000        0x8 ./MotorControl_Drivers/firmware/drivers/mss_nvm/mss_nvm.o
 .rodata.g_nvm32
                0x00000000        0x8 ./MotorControl_Drivers/firmware/drivers/mss_nvm/mss_nvm.o
 .bss.g_envm_ctrl_locks
                0x00000000        0x1 ./MotorControl_Drivers/firmware/drivers/mss_nvm/mss_nvm.o
 .text          0x00000000        0x0 ./MotorControl_Drivers/firmware/drivers/mss_hpdma/mss_hpdma.o
 .data          0x00000000        0x0 ./MotorControl_Drivers/firmware/drivers/mss_hpdma/mss_hpdma.o
 .bss           0x00000000        0x0 ./MotorControl_Drivers/firmware/drivers/mss_hpdma/mss_hpdma.o
 .text.MSS_HPDMA_init
                0x00000000       0x50 ./MotorControl_Drivers/firmware/drivers/mss_hpdma/mss_hpdma.o
 .text.MSS_HPDMA_pause
                0x00000000       0x10 ./MotorControl_Drivers/firmware/drivers/mss_hpdma/mss_hpdma.o
 .text.MSS_HPDMA_resume
                0x00000000       0x10 ./MotorControl_Drivers/firmware/drivers/mss_hpdma/mss_hpdma.o
 .text.MSS_HPDMA_abort
                0x00000000       0x10 ./MotorControl_Drivers/firmware/drivers/mss_hpdma/mss_hpdma.o
 .text.MSS_HPDMA_get_transfer_status
                0x00000000        0xc ./MotorControl_Drivers/firmware/drivers/mss_hpdma/mss_hpdma.o
 .text.MSS_HPDMA_set_handler
                0x00000000        0xc ./MotorControl_Drivers/firmware/drivers/mss_hpdma/mss_hpdma.o
 .text          0x00000000        0x0 ./MotorControl_Drivers/firmware/drivers/mss_gpio/mss_gpio.o
 .data          0x00000000        0x0 ./MotorControl_Drivers/firmware/drivers/mss_gpio/mss_gpio.o
 .bss           0x00000000        0x0 ./MotorControl_Drivers/firmware/drivers/mss_gpio/mss_gpio.o
 .text.MSS_GPIO_init
                0x00000000       0x60 ./MotorControl_Drivers/firmware/drivers/mss_gpio/mss_gpio.o
 .text.MSS_GPIO_config
                0x00000000       0x18 ./MotorControl_Drivers/firmware/drivers/mss_gpio/mss_gpio.o
 .text.MSS_GPIO_drive_inout
                0x00000000       0x5c ./MotorControl_Drivers/firmware/drivers/mss_gpio/mss_gpio.o
 .text.MSS_GPIO_enable_irq
                0x00000000       0x3c ./MotorControl_Drivers/firmware/drivers/mss_gpio/mss_gpio.o
 .text.MSS_GPIO_disable_irq
                0x00000000       0x1c ./MotorControl_Drivers/firmware/drivers/mss_gpio/mss_gpio.o
 .text.MSS_GPIO_clear_irq
                0x00000000       0x18 ./MotorControl_Drivers/firmware/drivers/mss_gpio/mss_gpio.o
 .rodata.g_gpio_irqn_lut
                0x00000000       0x20 ./MotorControl_Drivers/firmware/drivers/mss_gpio/mss_gpio.o
 .rodata.g_config_reg_lut
                0x00000000       0x80 ./MotorControl_Drivers/firmware/drivers/mss_gpio/mss_gpio.o
 .text          0x00000000        0x0 ./MotorControl_Drivers/firmware/CMSIS/startup_gcc/newlib_stubs.o
 .data          0x00000000        0x0 ./MotorControl_Drivers/firmware/CMSIS/startup_gcc/newlib_stubs.o
 .bss           0x00000000        0x0 ./MotorControl_Drivers/firmware/CMSIS/startup_gcc/newlib_stubs.o
 .text._close   0x00000000        0x6 ./MotorControl_Drivers/firmware/CMSIS/startup_gcc/newlib_stubs.o
 .text._execve  0x00000000       0x10 ./MotorControl_Drivers/firmware/CMSIS/startup_gcc/newlib_stubs.o
 .text._exit    0x00000000        0x2 ./MotorControl_Drivers/firmware/CMSIS/startup_gcc/newlib_stubs.o
 .text._fork    0x00000000       0x10 ./MotorControl_Drivers/firmware/CMSIS/startup_gcc/newlib_stubs.o
 .text._fstat   0x00000000        0xa ./MotorControl_Drivers/firmware/CMSIS/startup_gcc/newlib_stubs.o
 .text._getpid  0x00000000        0x4 ./MotorControl_Drivers/firmware/CMSIS/startup_gcc/newlib_stubs.o
 .text._isatty  0x00000000        0x4 ./MotorControl_Drivers/firmware/CMSIS/startup_gcc/newlib_stubs.o
 .text._kill    0x00000000       0x10 ./MotorControl_Drivers/firmware/CMSIS/startup_gcc/newlib_stubs.o
 .text._link    0x00000000       0x10 ./MotorControl_Drivers/firmware/CMSIS/startup_gcc/newlib_stubs.o
 .text._lseek   0x00000000        0x4 ./MotorControl_Drivers/firmware/CMSIS/startup_gcc/newlib_stubs.o
 .text._open    0x00000000        0x6 ./MotorControl_Drivers/firmware/CMSIS/startup_gcc/newlib_stubs.o
 .text._read    0x00000000        0x4 ./MotorControl_Drivers/firmware/CMSIS/startup_gcc/newlib_stubs.o
 .text._write_r
                0x00000000        0x4 ./MotorControl_Drivers/firmware/CMSIS/startup_gcc/newlib_stubs.o
 .text._sbrk    0x00000000       0x38 ./MotorControl_Drivers/firmware/CMSIS/startup_gcc/newlib_stubs.o
 .text._stat    0x00000000        0xa ./MotorControl_Drivers/firmware/CMSIS/startup_gcc/newlib_stubs.o
 .text._times   0x00000000        0x6 ./MotorControl_Drivers/firmware/CMSIS/startup_gcc/newlib_stubs.o
 .text._unlink  0x00000000       0x10 ./MotorControl_Drivers/firmware/CMSIS/startup_gcc/newlib_stubs.o
 .text._wait    0x00000000       0x10 ./MotorControl_Drivers/firmware/CMSIS/startup_gcc/newlib_stubs.o
 .data.environ  0x00000000        0x4 ./MotorControl_Drivers/firmware/CMSIS/startup_gcc/newlib_stubs.o
 .bss.__env     0x00000000        0x4 ./MotorControl_Drivers/firmware/CMSIS/startup_gcc/newlib_stubs.o
 .bss.heap_end.5162
                0x00000000        0x4 ./MotorControl_Drivers/firmware/CMSIS/startup_gcc/newlib_stubs.o
 .text          0x00000000        0x0 ./MotorControl_Drivers/firmware/CMSIS/startup_gcc/startup_m2sxxx.o
 .data          0x00000000        0x0 ./MotorControl_Drivers/firmware/CMSIS/startup_gcc/startup_m2sxxx.o
 .bss           0x00000000        0x0 ./MotorControl_Drivers/firmware/CMSIS/startup_gcc/startup_m2sxxx.o
 .text          0x00000000        0x0 ./MotorControl_Drivers/firmware/CMSIS/system_m2sxxx.o
 .data          0x00000000        0x0 ./MotorControl_Drivers/firmware/CMSIS/system_m2sxxx.o
 .bss           0x00000000        0x0 ./MotorControl_Drivers/firmware/CMSIS/system_m2sxxx.o
 .text.set_clock_frequency_globals
                0x00000000       0x40 ./MotorControl_Drivers/firmware/CMSIS/system_m2sxxx.o
 .text.SystemCoreClockUpdate
                0x00000000       0xac ./MotorControl_Drivers/firmware/CMSIS/system_m2sxxx.o
 .rodata        0x00000000        0x8 ./MotorControl_Drivers/firmware/CMSIS/system_m2sxxx.o
 .data.g_FrequencyFIC64
                0x00000000        0x4 ./MotorControl_Drivers/firmware/CMSIS/system_m2sxxx.o
 .data.g_FrequencyPCLK2
                0x00000000        0x4 ./MotorControl_Drivers/firmware/CMSIS/system_m2sxxx.o
 .data.g_FrequencyFIC0
                0x00000000        0x4 ./MotorControl_Drivers/firmware/CMSIS/system_m2sxxx.o
 .data.g_FrequencyFIC1
                0x00000000        0x4 ./MotorControl_Drivers/firmware/CMSIS/system_m2sxxx.o
 .data.g_FrequencyPCLK0
                0x00000000        0x4 ./MotorControl_Drivers/firmware/CMSIS/system_m2sxxx.o
 .data.g_FrequencyPCLK1
                0x00000000        0x4 ./MotorControl_Drivers/firmware/CMSIS/system_m2sxxx.o
 .data.SystemCoreClock
                0x00000000        0x4 ./MotorControl_Drivers/firmware/CMSIS/system_m2sxxx.o
 .text          0x00000000        0x0 ./MotorControl_App/MCCalc.o
 .data          0x00000000        0x0 ./MotorControl_App/MCCalc.o
 .bss           0x00000000        0x0 ./MotorControl_App/MCCalc.o
 .text          0x00000000        0x0 ./MotorControl_App/MCFPGAIF.o
 .data          0x00000000        0x0 ./MotorControl_App/MCFPGAIF.o
 .bss           0x00000000        0x0 ./MotorControl_App/MCFPGAIF.o
 .text          0x00000000        0x0 ./MotorControl_App/USBMsgHandler.o
 .data          0x00000000        0x0 ./MotorControl_App/USBMsgHandler.o
 .bss           0x00000000        0x0 ./MotorControl_App/USBMsgHandler.o
 COMMON         0x00000000        0x4 ./MotorControl_App/USBMsgHandler.o
 .text          0x00000000        0x0 ./MotorControl_App/main.o
 .data          0x00000000        0x0 ./MotorControl_App/main.o
 .bss           0x00000000        0x0 ./MotorControl_App/main.o
 .text          0x00000000        0x0 ./MotorControl_App/usb_user_descriptors.o
 .data          0x00000000        0x0 ./MotorControl_App/usb_user_descriptors.o
 .bss           0x00000000        0x0 ./MotorControl_App/usb_user_descriptors.o
 .text          0x00000000        0x0 f:/microsemi/softconsole_v4.0/arm-none-eabi-gcc/bin/../lib/gcc/arm-none-eabi/4.9.3/../../../../arm-none-eabi/lib/armv7-m\libg_nano.a(lib_a-errno.o)
 .data          0x00000000        0x0 f:/microsemi/softconsole_v4.0/arm-none-eabi-gcc/bin/../lib/gcc/arm-none-eabi/4.9.3/../../../../arm-none-eabi/lib/armv7-m\libg_nano.a(lib_a-errno.o)
 .bss           0x00000000        0x0 f:/microsemi/softconsole_v4.0/arm-none-eabi-gcc/bin/../lib/gcc/arm-none-eabi/4.9.3/../../../../arm-none-eabi/lib/armv7-m\libg_nano.a(lib_a-errno.o)
 .text.__errno  0x00000000        0xc f:/microsemi/softconsole_v4.0/arm-none-eabi-gcc/bin/../lib/gcc/arm-none-eabi/4.9.3/../../../../arm-none-eabi/lib/armv7-m\libg_nano.a(lib_a-errno.o)
 .text          0x00000000        0x0 f:/microsemi/softconsole_v4.0/arm-none-eabi-gcc/bin/../lib/gcc/arm-none-eabi/4.9.3/../../../../arm-none-eabi/lib/armv7-m\libg_nano.a(lib_a-exit.o)
 .data          0x00000000        0x0 f:/microsemi/softconsole_v4.0/arm-none-eabi-gcc/bin/../lib/gcc/arm-none-eabi/4.9.3/../../../../arm-none-eabi/lib/armv7-m\libg_nano.a(lib_a-exit.o)
 .bss           0x00000000        0x0 f:/microsemi/softconsole_v4.0/arm-none-eabi-gcc/bin/../lib/gcc/arm-none-eabi/4.9.3/../../../../arm-none-eabi/lib/armv7-m\libg_nano.a(lib_a-exit.o)
 .text.exit     0x00000000       0x28 f:/microsemi/softconsole_v4.0/arm-none-eabi-gcc/bin/../lib/gcc/arm-none-eabi/4.9.3/../../../../arm-none-eabi/lib/armv7-m\libg_nano.a(lib_a-exit.o)
 .text          0x00000000        0x0 f:/microsemi/softconsole_v4.0/arm-none-eabi-gcc/bin/../lib/gcc/arm-none-eabi/4.9.3/../../../../arm-none-eabi/lib/armv7-m\libg_nano.a(lib_a-impure.o)
 .data          0x00000000        0x0 f:/microsemi/softconsole_v4.0/arm-none-eabi-gcc/bin/../lib/gcc/arm-none-eabi/4.9.3/../../../../arm-none-eabi/lib/armv7-m\libg_nano.a(lib_a-impure.o)
 .bss           0x00000000        0x0 f:/microsemi/softconsole_v4.0/arm-none-eabi-gcc/bin/../lib/gcc/arm-none-eabi/4.9.3/../../../../arm-none-eabi/lib/armv7-m\libg_nano.a(lib_a-impure.o)
 .data.impure_data
                0x00000000       0x60 f:/microsemi/softconsole_v4.0/arm-none-eabi-gcc/bin/../lib/gcc/arm-none-eabi/4.9.3/../../../../arm-none-eabi/lib/armv7-m\libg_nano.a(lib_a-impure.o)
 .data._impure_ptr
                0x00000000        0x4 f:/microsemi/softconsole_v4.0/arm-none-eabi-gcc/bin/../lib/gcc/arm-none-eabi/4.9.3/../../../../arm-none-eabi/lib/armv7-m\libg_nano.a(lib_a-impure.o)
 .rodata.str1.1
                0x00000000        0x2 f:/microsemi/softconsole_v4.0/arm-none-eabi-gcc/bin/../lib/gcc/arm-none-eabi/4.9.3/../../../../arm-none-eabi/lib/armv7-m\libg_nano.a(lib_a-impure.o)
 .rodata._global_impure_ptr
                0x00000000        0x4 f:/microsemi/softconsole_v4.0/arm-none-eabi-gcc/bin/../lib/gcc/arm-none-eabi/4.9.3/../../../../arm-none-eabi/lib/armv7-m\libg_nano.a(lib_a-impure.o)
 .text          0x00000000        0x0 f:/microsemi/softconsole_v4.0/arm-none-eabi-gcc/bin/../lib/gcc/arm-none-eabi/4.9.3/../../../../arm-none-eabi/lib/armv7-m\libg_nano.a(lib_a-init.o)
 .data          0x00000000        0x0 f:/microsemi/softconsole_v4.0/arm-none-eabi-gcc/bin/../lib/gcc/arm-none-eabi/4.9.3/../../../../arm-none-eabi/lib/armv7-m\libg_nano.a(lib_a-init.o)
 .bss           0x00000000        0x0 f:/microsemi/softconsole_v4.0/arm-none-eabi-gcc/bin/../lib/gcc/arm-none-eabi/4.9.3/../../../../arm-none-eabi/lib/armv7-m\libg_nano.a(lib_a-init.o)
 .text          0x00000000        0x0 f:/microsemi/softconsole_v4.0/arm-none-eabi-gcc/bin/../lib/gcc/arm-none-eabi/4.9.3/../../../../arm-none-eabi/lib/armv7-m\libg_nano.a(lib_a-memcpy.o)
 .data          0x00000000        0x0 f:/microsemi/softconsole_v4.0/arm-none-eabi-gcc/bin/../lib/gcc/arm-none-eabi/4.9.3/../../../../arm-none-eabi/lib/armv7-m\libg_nano.a(lib_a-memcpy.o)
 .bss           0x00000000        0x0 f:/microsemi/softconsole_v4.0/arm-none-eabi-gcc/bin/../lib/gcc/arm-none-eabi/4.9.3/../../../../arm-none-eabi/lib/armv7-m\libg_nano.a(lib_a-memcpy.o)
 .text.memcpy   0x00000000       0x16 f:/microsemi/softconsole_v4.0/arm-none-eabi-gcc/bin/../lib/gcc/arm-none-eabi/4.9.3/../../../../arm-none-eabi/lib/armv7-m\libg_nano.a(lib_a-memcpy.o)
 .text          0x00000000        0x0 f:/microsemi/softconsole_v4.0/arm-none-eabi-gcc/bin/../lib/gcc/arm-none-eabi/4.9.3/../../../../arm-none-eabi/lib/armv7-m\libg_nano.a(lib_a-memset.o)
 .data          0x00000000        0x0 f:/microsemi/softconsole_v4.0/arm-none-eabi-gcc/bin/../lib/gcc/arm-none-eabi/4.9.3/../../../../arm-none-eabi/lib/armv7-m\libg_nano.a(lib_a-memset.o)
 .bss           0x00000000        0x0 f:/microsemi/softconsole_v4.0/arm-none-eabi-gcc/bin/../lib/gcc/arm-none-eabi/4.9.3/../../../../arm-none-eabi/lib/armv7-m\libg_nano.a(lib_a-memset.o)
 .text.memset   0x00000000       0x10 f:/microsemi/softconsole_v4.0/arm-none-eabi-gcc/bin/../lib/gcc/arm-none-eabi/4.9.3/../../../../arm-none-eabi/lib/armv7-m\libg_nano.a(lib_a-memset.o)
 .text          0x00000000        0x0 f:/microsemi/softconsole_v4.0/arm-none-eabi-gcc/bin/../lib/gcc/arm-none-eabi/4.9.3/armv7-m/crtend.o
 .data          0x00000000        0x0 f:/microsemi/softconsole_v4.0/arm-none-eabi-gcc/bin/../lib/gcc/arm-none-eabi/4.9.3/armv7-m/crtend.o
 .bss           0x00000000        0x0 f:/microsemi/softconsole_v4.0/arm-none-eabi-gcc/bin/../lib/gcc/arm-none-eabi/4.9.3/armv7-m/crtend.o
 .eh_frame      0x00000000        0x4 f:/microsemi/softconsole_v4.0/arm-none-eabi-gcc/bin/../lib/gcc/arm-none-eabi/4.9.3/armv7-m/crtend.o
 .text          0x00000000        0x0 f:/microsemi/softconsole_v4.0/arm-none-eabi-gcc/bin/../lib/gcc/arm-none-eabi/4.9.3/armv7-m/crtn.o
 .data          0x00000000        0x0 f:/microsemi/softconsole_v4.0/arm-none-eabi-gcc/bin/../lib/gcc/arm-none-eabi/4.9.3/armv7-m/crtn.o
 .bss           0x00000000        0x0 f:/microsemi/softconsole_v4.0/arm-none-eabi-gcc/bin/../lib/gcc/arm-none-eabi/4.9.3/armv7-m/crtn.o

Memory Configuration

Name             Origin             Length             Attributes
rom              0x00000000         0x00040000         xr
ram              0x20000000         0x00010000         xrw
*default*        0x00000000         0xffffffff

Linker script and memory map

LOAD f:/microsemi/softconsole_v4.0/arm-none-eabi-gcc/bin/../lib/gcc/arm-none-eabi/4.9.3/armv7-m/crti.o
LOAD f:/microsemi/softconsole_v4.0/arm-none-eabi-gcc/bin/../lib/gcc/arm-none-eabi/4.9.3/armv7-m/crtbegin.o
LOAD f:/microsemi/softconsole_v4.0/arm-none-eabi-gcc/bin/../lib/gcc/arm-none-eabi/4.9.3/../../../../arm-none-eabi/lib/armv7-m/crt0.o
LOAD ./MotorControl_Drivers/firmware/hal/CortexM3/GNU/hal.o
LOAD ./MotorControl_Drivers/firmware/hal/CortexM3/GNU/hw_reg_access.o
LOAD ./MotorControl_Drivers/firmware/hal/CortexM3/cortex_nvic.o
LOAD ./MotorControl_Drivers/firmware/drivers_config/sys_config/sys_config.o
LOAD ./MotorControl_Drivers/firmware/drivers/mss_usb/mss_usb_common_cif.o
LOAD ./MotorControl_Drivers/firmware/drivers/mss_usb/mss_usb_device.o
LOAD ./MotorControl_Drivers/firmware/drivers/mss_usb/mss_usb_device_cdc.o
LOAD ./MotorControl_Drivers/firmware/drivers/mss_usb/mss_usb_device_cif.o
LOAD ./MotorControl_Drivers/firmware/drivers/mss_usb/mss_usb_device_hid.o
LOAD ./MotorControl_Drivers/firmware/drivers/mss_usb/mss_usb_device_msd.o
LOAD ./MotorControl_Drivers/firmware/drivers/mss_usb/mss_usb_device_printer.o
LOAD ./MotorControl_Drivers/firmware/drivers/mss_usb/mss_usb_device_vendor.o
LOAD ./MotorControl_Drivers/firmware/drivers/mss_usb/mss_usb_host.o
LOAD ./MotorControl_Drivers/firmware/drivers/mss_usb/mss_usb_host_cif.o
LOAD ./MotorControl_Drivers/firmware/drivers/mss_usb/mss_usb_host_msc.o
LOAD ./MotorControl_Drivers/firmware/drivers/mss_sys_services/mss_comblk.o
LOAD ./MotorControl_Drivers/firmware/drivers/mss_sys_services/mss_sys_services.o
LOAD ./MotorControl_Drivers/firmware/drivers/mss_nvm/mss_nvm.o
LOAD ./MotorControl_Drivers/firmware/drivers/mss_hpdma/mss_hpdma.o
LOAD ./MotorControl_Drivers/firmware/drivers/mss_gpio/mss_gpio.o
LOAD ./MotorControl_Drivers/firmware/CMSIS/startup_gcc/newlib_stubs.o
LOAD ./MotorControl_Drivers/firmware/CMSIS/startup_gcc/startup_m2sxxx.o
LOAD ./MotorControl_Drivers/firmware/CMSIS/system_m2sxxx.o
LOAD ./MotorControl_App/MCCalc.o
LOAD ./MotorControl_App/MCFPGAIF.o
LOAD ./MotorControl_App/USBMsgHandler.o
LOAD ./MotorControl_App/main.o
LOAD ./MotorControl_App/usb_user_descriptors.o
START GROUP
LOAD f:/microsemi/softconsole_v4.0/arm-none-eabi-gcc/bin/../lib/gcc/arm-none-eabi/4.9.3/armv7-m\libgcc.a
LOAD f:/microsemi/softconsole_v4.0/arm-none-eabi-gcc/bin/../lib/gcc/arm-none-eabi/4.9.3/../../../../arm-none-eabi/lib/armv7-m\libg_nano.a
LOAD f:/microsemi/softconsole_v4.0/arm-none-eabi-gcc/bin/../lib/gcc/arm-none-eabi/4.9.3/../../../../arm-none-eabi/lib/armv7-m\libc_nano.a
END GROUP
START GROUP
LOAD f:/microsemi/softconsole_v4.0/arm-none-eabi-gcc/bin/../lib/gcc/arm-none-eabi/4.9.3/armv7-m\libgcc.a
LOAD f:/microsemi/softconsole_v4.0/arm-none-eabi-gcc/bin/../lib/gcc/arm-none-eabi/4.9.3/../../../../arm-none-eabi/lib/armv7-m\libc_nano.a
END GROUP
LOAD f:/microsemi/softconsole_v4.0/arm-none-eabi-gcc/bin/../lib/gcc/arm-none-eabi/4.9.3/armv7-m/crtend.o
LOAD f:/microsemi/softconsole_v4.0/arm-none-eabi-gcc/bin/../lib/gcc/arm-none-eabi/4.9.3/armv7-m/crtn.o
START GROUP
LOAD f:/microsemi/softconsole_v4.0/arm-none-eabi-gcc/bin/../lib/gcc/arm-none-eabi/4.9.3/../../../../arm-none-eabi/lib/armv7-m\libc.a
LOAD f:/microsemi/softconsole_v4.0/arm-none-eabi-gcc/bin/../lib/gcc/arm-none-eabi/4.9.3/armv7-m\libgcc.a
LOAD f:/microsemi/softconsole_v4.0/arm-none-eabi-gcc/bin/../lib/gcc/arm-none-eabi/4.9.3/../../../../arm-none-eabi/lib/armv7-m\libm.a
END GROUP
                0x00000000                __DYNAMIC = 0x0
                0x20000000                RAM_START_ADDRESS = 0x20000000
                0x00010000                RAM_SIZE = 0x10000
                0x00001000                MAIN_STACK_SIZE = 0x1000
                0x00001000                MIN_SIZE_HEAP = 0x1000
                0x20010000                PROVIDE (__main_stack_start, (RAM_START_ADDRESS + RAM_SIZE))
                0x2000f000                PROVIDE (__process_stack_start, (__main_stack_start - MAIN_STACK_SIZE))
                0x20010000                PROVIDE (_estack, __main_stack_start)
                0x00000000                PROVIDE (__mirrored_nvm, 0x0)
                0x00000000                PROVIDE (__smartfusion2_memory_remap, 0x0)

.vector_table   0x00000000      0x190
                0x00000000                __vector_table_load = LOADADDR (.vector_table)
                0x00000000                __vector_table_start = .
                0x00000000                __vector_table_vma_base_address = .
 *(.isr_vector)
 .isr_vector    0x00000000      0x190 ./MotorControl_Drivers/firmware/CMSIS/startup_gcc/startup_m2sxxx.o
                0x00000000                g_pfnVectors
                0x00000190                . = ALIGN (0x10)
                0x00000190                _evector_table = .

.boot_code      0x00000190      0x330
 *(.boot_code)
 .boot_code     0x00000190      0x324 ./MotorControl_Drivers/firmware/CMSIS/startup_gcc/startup_m2sxxx.o
                0x00000190                Reset_Handler
                0x0000037e                NMI_Handler
                0x00000380                HardFault_Handler
                0x00000382                MemManage_Handler
                0x00000384                BusFault_Handler
                0x00000386                UsageFault_Handler
                0x00000388                SVC_Handler
                0x0000038a                DebugMon_Handler
                0x0000038c                PendSV_Handler
                0x0000038e                SysTick_Handler
                0x00000390                WdogWakeup_IRQHandler
                0x00000392                RTC_Wakeup_IRQHandler
                0x00000394                SPI0_IRQHandler
                0x00000396                SPI1_IRQHandler
                0x00000398                I2C0_IRQHandler
                0x0000039a                I2C0_SMBAlert_IRQHandler
                0x0000039c                I2C0_SMBus_IRQHandler
                0x0000039e                I2C1_IRQHandler
                0x000003a0                I2C1_SMBAlert_IRQHandler
                0x000003a2                I2C1_SMBus_IRQHandler
                0x000003a4                UART0_IRQHandler
                0x000003a6                UART1_IRQHandler
                0x000003a8                EthernetMAC_IRQHandler
                0x000003aa                DMA_IRQHandler
                0x000003ac                Timer1_IRQHandler
                0x000003ae                Timer2_IRQHandler
                0x000003b0                CAN_IRQHandler
                0x000003b2                ENVM0_IRQHandler
                0x000003b4                ENVM1_IRQHandler
                0x000003bc                PLL_Lock_IRQHandler
                0x000003be                PLL_LockLost_IRQHandler
                0x000003c0                CommSwitchError_IRQHandler
                0x000003c2                CacheError_IRQHandler
                0x000003c4                DDR_IRQHandler
                0x000003ca                ECC_Error_IRQHandler
                0x000003cc                MDDR_IOCalib_IRQHandler
                0x000003ce                FAB_PLL_Lock_IRQHandler
                0x000003d0                FAB_PLL_LockLost_IRQHandler
                0x000003d2                FIC64_IRQHandler
                0x000003d4                FabricIrq0_IRQHandler
                0x000003d6                FabricIrq1_IRQHandler
                0x000003d8                FabricIrq2_IRQHandler
                0x000003da                FabricIrq3_IRQHandler
                0x000003dc                FabricIrq4_IRQHandler
                0x000003de                FabricIrq5_IRQHandler
                0x000003e0                FabricIrq6_IRQHandler
                0x000003e2                FabricIrq7_IRQHandler
                0x000003e4                FabricIrq8_IRQHandler
                0x000003e6                FabricIrq9_IRQHandler
                0x000003e8                FabricIrq10_IRQHandler
                0x000003ea                FabricIrq11_IRQHandler
                0x000003ec                FabricIrq12_IRQHandler
                0x000003ee                FabricIrq13_IRQHandler
                0x000003f0                FabricIrq14_IRQHandler
                0x000003f2                FabricIrq15_IRQHandler
                0x000003f4                GPIO0_IRQHandler
                0x000003f6                GPIO1_IRQHandler
                0x000003f8                GPIO2_IRQHandler
                0x000003fa                GPIO3_IRQHandler
                0x000003fc                GPIO4_IRQHandler
                0x000003fe                GPIO5_IRQHandler
                0x00000400                GPIO6_IRQHandler
                0x00000402                GPIO7_IRQHandler
                0x00000404                GPIO8_IRQHandler
                0x00000406                GPIO9_IRQHandler
                0x00000408                GPIO10_IRQHandler
                0x0000040a                GPIO11_IRQHandler
                0x0000040c                GPIO12_IRQHandler
                0x0000040e                GPIO13_IRQHandler
                0x00000410                GPIO14_IRQHandler
                0x00000412                GPIO15_IRQHandler
                0x00000414                GPIO16_IRQHandler
                0x00000416                GPIO17_IRQHandler
                0x00000418                GPIO18_IRQHandler
                0x0000041a                GPIO19_IRQHandler
                0x0000041c                GPIO20_IRQHandler
                0x0000041e                GPIO21_IRQHandler
                0x00000420                GPIO22_IRQHandler
                0x00000422                GPIO23_IRQHandler
                0x00000424                GPIO24_IRQHandler
                0x00000426                GPIO25_IRQHandler
                0x00000428                GPIO26_IRQHandler
                0x0000042a                GPIO27_IRQHandler
                0x0000042c                GPIO28_IRQHandler
                0x0000042e                GPIO29_IRQHandler
                0x00000430                GPIO30_IRQHandler
                0x00000432                GPIO31_IRQHandler
                0x00000434                mscc_post_hw_cfg_init
                0x000004c0                . = ALIGN (0x10)
 *fill*         0x000004b4        0xc 

.text           0x000004c0     0x3010
 CREATE_OBJECT_SYMBOLS
                0x000004c0                __text_load = LOADADDR (.text)
                0x000004c0                __text_start = .
 *(.text .text.* .gnu.linkonce.t.*)
 .text          0x000004c0       0x5c f:/microsemi/softconsole_v4.0/arm-none-eabi-gcc/bin/../lib/gcc/arm-none-eabi/4.9.3/armv7-m/crtbegin.o
 .text          0x0000051c       0x90 ./MotorControl_Drivers/firmware/hal/CortexM3/GNU/hw_reg_access.o
                0x0000051c                HW_set_32bit_reg
                0x00000520                HW_get_32bit_reg
                0x00000524                HW_set_32bit_reg_field
                0x00000540                HW_get_32bit_reg_field
                0x0000054c                HW_set_16bit_reg
                0x00000550                HW_get_16bit_reg
                0x00000554                HW_set_16bit_reg_field
                0x00000570                HW_get_16bit_reg_field
                0x0000057c                HW_set_8bit_reg
                0x00000580                HW_get_8bit_reg
                0x00000584                HW_set_8bit_reg_field
                0x000005a0                HW_get_8bit_reg_field
 .text.MSS_USB_CIF_rx_ep_disable_irq
                0x000005ac       0x18 ./MotorControl_Drivers/firmware/drivers/mss_usb/mss_usb_common_cif.o
 .text.MSS_USB_CIF_read_rx_fifo
                0x000005c4       0x40 ./MotorControl_Drivers/firmware/drivers/mss_usb/mss_usb_common_cif.o
 .text.USB_IRQHandler
                0x00000604      0x394 ./MotorControl_Drivers/firmware/drivers/mss_usb/mss_usb_common_cif.o
                0x00000604                USB_IRQHandler
 .text.USB_DMA_IRQHandler
                0x00000998      0x1fc ./MotorControl_Drivers/firmware/drivers/mss_usb/mss_usb_common_cif.o
                0x00000998                USB_DMA_IRQHandler
 .text.MSS_USB_CIF_ep_write_pkt
                0x00000b94      0x11c ./MotorControl_Drivers/firmware/drivers/mss_usb/mss_usb_common_cif.o
                0x00000b94                MSS_USB_CIF_ep_write_pkt
 .text.MSS_USB_CIF_configure_ep_dma
                0x00000cb0       0x5a ./MotorControl_Drivers/firmware/drivers/mss_usb/mss_usb_common_cif.o
                0x00000cb0                MSS_USB_CIF_configure_ep_dma
 *fill*         0x00000d0a        0x2 
 .text.MSS_USB_CIF_tx_ep_configure
                0x00000d0c      0x144 ./MotorControl_Drivers/firmware/drivers/mss_usb/mss_usb_common_cif.o
                0x00000d0c                MSS_USB_CIF_tx_ep_configure
 .text.MSS_USB_CIF_rx_ep_configure
                0x00000e50      0x154 ./MotorControl_Drivers/firmware/drivers/mss_usb/mss_usb_common_cif.o
                0x00000e50                MSS_USB_CIF_rx_ep_configure
 .text.MSS_USBD_sof_cb
                0x00000fa4        0x2 ./MotorControl_Drivers/firmware/drivers/mss_usb/mss_usb_device.o
 *fill*         0x00000fa6        0x2 
 .text.MSS_USBD_suspend_cb
                0x00000fa8       0x20 ./MotorControl_Drivers/firmware/drivers/mss_usb/mss_usb_device.o
 .text.MSS_USBD_resume_cb
                0x00000fc8        0xc ./MotorControl_Drivers/firmware/drivers/mss_usb/mss_usb_device.o
 .text.MSS_USBD_ep_datain_cb
                0x00000fd4       0x94 ./MotorControl_Drivers/firmware/drivers/mss_usb/mss_usb_device.o
 .text.MSS_USBD_ep_dataout_cb
                0x00001068       0xa8 ./MotorControl_Drivers/firmware/drivers/mss_usb/mss_usb_device.o
 .text.MSS_USBD_init
                0x00001110       0x40 ./MotorControl_Drivers/firmware/drivers/mss_usb/mss_usb_device.o
                0x00001110                MSS_USBD_init
 .text.MSS_USBD_set_descr_cb_handler
                0x00001150        0xc ./MotorControl_Drivers/firmware/drivers/mss_usb/mss_usb_device.o
                0x00001150                MSS_USBD_set_descr_cb_handler
 .text.MSS_USBD_set_class_cb_handler
                0x0000115c        0xc ./MotorControl_Drivers/firmware/drivers/mss_usb/mss_usb_device.o
                0x0000115c                MSS_USBD_set_class_cb_handler
 .text.MSS_USBD_tx_ep_flush_fifo
                0x00001168       0x1a ./MotorControl_Drivers/firmware/drivers/mss_usb/mss_usb_device.o
                0x00001168                MSS_USBD_tx_ep_flush_fifo
 .text.MSS_USBD_rx_ep_flush_fifo
                0x00001182       0x1a ./MotorControl_Drivers/firmware/drivers/mss_usb/mss_usb_device.o
                0x00001182                MSS_USBD_rx_ep_flush_fifo
 .text.MSS_USBD_cep_configure
                0x0000119c       0x20 ./MotorControl_Drivers/firmware/drivers/mss_usb/mss_usb_device.o
                0x0000119c                MSS_USBD_cep_configure
 .text.MSS_USBD_cep_read_prepare
                0x000011bc       0x20 ./MotorControl_Drivers/firmware/drivers/mss_usb/mss_usb_device.o
                0x000011bc                MSS_USBD_cep_read_prepare
 .text.MSS_USBD_reset_cb
                0x000011dc       0x58 ./MotorControl_Drivers/firmware/drivers/mss_usb/mss_usb_device.o
 .text.MSS_USBD_cep_datain_cb
                0x00001234       0x9c ./MotorControl_Drivers/firmware/drivers/mss_usb/mss_usb_device.o
 .text.MSS_USBD_cep_dataout_cb
                0x000012d0       0xb8 ./MotorControl_Drivers/firmware/drivers/mss_usb/mss_usb_device.o
 .text.MSS_USBD_cep_write
                0x00001388       0x20 ./MotorControl_Drivers/firmware/drivers/mss_usb/mss_usb_device.o
                0x00001388                MSS_USBD_cep_write
 .text.MSS_USBD_cep_setup_cb
                0x000013a8      0x51c ./MotorControl_Drivers/firmware/drivers/mss_usb/mss_usb_device.o
 .text.MSS_USBD_tx_ep_configure
                0x000018c4       0xd0 ./MotorControl_Drivers/firmware/drivers/mss_usb/mss_usb_device.o
                0x000018c4                MSS_USBD_tx_ep_configure
 .text.MSS_USBD_rx_ep_configure
                0x00001994       0xd0 ./MotorControl_Drivers/firmware/drivers/mss_usb/mss_usb_device.o
                0x00001994                MSS_USBD_rx_ep_configure
 .text.MSS_USBD_rx_ep_read_prepare
                0x00001a64       0x38 ./MotorControl_Drivers/firmware/drivers/mss_usb/mss_usb_device.o
                0x00001a64                MSS_USBD_rx_ep_read_prepare
 .text.MSS_USBD_tx_ep_write
                0x00001a9c       0x70 ./MotorControl_Drivers/firmware/drivers/mss_usb/mss_usb_device.o
                0x00001a9c                MSS_USBD_tx_ep_write
 .text.MSS_USBD_CIF_init
                0x00001b0c       0x54 ./MotorControl_Drivers/firmware/drivers/mss_usb/mss_usb_device_cif.o
                0x00001b0c                MSS_USBD_CIF_init
 .text.MSS_USBD_CIF_tx_ep_configure
                0x00001b60       0xa2 ./MotorControl_Drivers/firmware/drivers/mss_usb/mss_usb_device_cif.o
                0x00001b60                MSS_USBD_CIF_tx_ep_configure
 .text.MSS_USBD_CIF_rx_ep_configure
                0x00001c02       0xd2 ./MotorControl_Drivers/firmware/drivers/mss_usb/mss_usb_device_cif.o
                0x00001c02                MSS_USBD_CIF_rx_ep_configure
 .text.MSS_USBD_CIF_cep_configure
                0x00001cd4       0x18 ./MotorControl_Drivers/firmware/drivers/mss_usb/mss_usb_device_cif.o
                0x00001cd4                MSS_USBD_CIF_cep_configure
 .text.MSS_USBD_CIF_cep_rx_prepare
                0x00001cec       0x20 ./MotorControl_Drivers/firmware/drivers/mss_usb/mss_usb_device_cif.o
                0x00001cec                MSS_USBD_CIF_cep_rx_prepare
 .text.MSS_USBD_CIF_rx_ep_read_prepare
                0x00001d0c       0xcc ./MotorControl_Drivers/firmware/drivers/mss_usb/mss_usb_device_cif.o
                0x00001d0c                MSS_USBD_CIF_rx_ep_read_prepare
 .text.MSS_USBD_CIF_cep_write_pkt
                0x00001dd8       0x74 ./MotorControl_Drivers/firmware/drivers/mss_usb/mss_usb_device_cif.o
                0x00001dd8                MSS_USBD_CIF_cep_write_pkt
 .text.MSS_USBD_CIF_cep_read_pkt
                0x00001e4c       0x70 ./MotorControl_Drivers/firmware/drivers/mss_usb/mss_usb_device_cif.o
                0x00001e4c                MSS_USBD_CIF_cep_read_pkt
 .text.USBD_HID_deinit_cb
                0x00001ebc       0x10 ./MotorControl_Drivers/firmware/drivers/mss_usb/mss_usb_device_hid.o
                0x00001ebc                USBD_HID_deinit_cb
 .text.USBD_HID_process_request_cb
                0x00001ecc        0x4 ./MotorControl_Drivers/firmware/drivers/mss_usb/mss_usb_device_hid.o
                0x00001ecc                USBD_HID_process_request_cb
 .text.USBD_HID_cep_datain_cb
                0x00001ed0        0x4 ./MotorControl_Drivers/firmware/drivers/mss_usb/mss_usb_device_hid.o
                0x00001ed0                USBD_HID_cep_datain_cb
 .text.USBD_HID_cep_dataout_cb
                0x00001ed4        0x4 ./MotorControl_Drivers/firmware/drivers/mss_usb/mss_usb_device_hid.o
                0x00001ed4                USBD_HID_cep_dataout_cb
 .text.USBD_HID_init_cb
                0x00001ed8       0x38 ./MotorControl_Drivers/firmware/drivers/mss_usb/mss_usb_device_hid.o
                0x00001ed8                USBD_HID_init_cb
 .text.USBD_HID_data_in_cb
                0x00001f10       0x1c ./MotorControl_Drivers/firmware/drivers/mss_usb/mss_usb_device_hid.o
                0x00001f10                USBD_HID_data_in_cb
 .text.USBD_HID_get_descriptor_cb
                0x00001f2c       0x40 ./MotorControl_Drivers/firmware/drivers/mss_usb/mss_usb_device_hid.o
                0x00001f2c                USBD_HID_get_descriptor_cb
 .text.MSS_USBD_HID_tx_report
                0x00001f6c       0x2c ./MotorControl_Drivers/firmware/drivers/mss_usb/mss_usb_device_hid.o
                0x00001f6c                MSS_USBD_HID_tx_report
 .text.MSS_USBD_HID_rx_report
                0x00001f98       0x24 ./MotorControl_Drivers/firmware/drivers/mss_usb/mss_usb_device_hid.o
                0x00001f98                MSS_USBD_HID_rx_report
 .text.USBD_HID_dataout_cb
                0x00001fbc       0x28 ./MotorControl_Drivers/firmware/drivers/mss_usb/mss_usb_device_hid.o
                0x00001fbc                USBD_HID_dataout_cb
 .text.MSS_USBD_HID_tx_done
                0x00001fe4        0xc ./MotorControl_Drivers/firmware/drivers/mss_usb/mss_usb_device_hid.o
                0x00001fe4                MSS_USBD_HID_tx_done
 .text.MSS_USBD_HID_init
                0x00001ff0       0x14 ./MotorControl_Drivers/firmware/drivers/mss_usb/mss_usb_device_hid.o
                0x00001ff0                MSS_USBD_HID_init
 .text.complete_request
                0x00002004       0x28 ./MotorControl_Drivers/firmware/drivers/mss_sys_services/mss_comblk.o
 .text.fill_tx_fifo
                0x0000202c       0x40 ./MotorControl_Drivers/firmware/drivers/mss_sys_services/mss_comblk.o
 .text.process_sys_ctrl_command
                0x0000206c       0x10 ./MotorControl_Drivers/firmware/drivers/mss_sys_services/mss_comblk.o
 .text.abort_current_cmd
                0x0000207c       0x30 ./MotorControl_Drivers/firmware/drivers/mss_sys_services/mss_comblk.o
 .text.ComBlk_IRQHandler
                0x000020ac      0x228 ./MotorControl_Drivers/firmware/drivers/mss_sys_services/mss_comblk.o
                0x000020ac                ComBlk_IRQHandler
 .text.MSS_HPDMA_start
                0x000022d4       0x94 ./MotorControl_Drivers/firmware/drivers/mss_hpdma/mss_hpdma.o
                0x000022d4                MSS_HPDMA_start
 .text.HPDMA_Complete_IRQHandler
                0x00002368       0x3c ./MotorControl_Drivers/firmware/drivers/mss_hpdma/mss_hpdma.o
                0x00002368                HPDMA_Complete_IRQHandler
 .text.HPDMA_Error_IRQHandler
                0x000023a4       0x78 ./MotorControl_Drivers/firmware/drivers/mss_hpdma/mss_hpdma.o
                0x000023a4                HPDMA_Error_IRQHandler
 .text.MSS_GPIO_set_output
                0x0000241c       0x2c ./MotorControl_Drivers/firmware/drivers/mss_gpio/mss_gpio.o
                0x0000241c                MSS_GPIO_set_output
 .text.SystemInit
                0x00002448       0x40 ./MotorControl_Drivers/firmware/CMSIS/system_m2sxxx.o
                0x00002448                SystemInit
 .text.MC_StepperInit
                0x00002488       0x34 ./MotorControl_App/MCCalc.o
                0x00002488                MC_StepperInit
 .text.MC_StepperConstCal
                0x000024bc       0x58 ./MotorControl_App/MCCalc.o
                0x000024bc                MC_StepperConstCal
 .text.MC_BLDCInit
                0x00002514       0x88 ./MotorControl_App/MCCalc.o
                0x00002514                MC_BLDCInit
 .text.MC_BLDCConstCal
                0x0000259c      0x10c ./MotorControl_App/MCCalc.o
                0x0000259c                MC_BLDCConstCal
 .text.MotorControl_Start
                0x000026a8       0x28 ./MotorControl_App/MCFPGAIF.o
                0x000026a8                MotorControl_Start
 .text.MotorControl_Stop
                0x000026d0       0x38 ./MotorControl_App/MCFPGAIF.o
                0x000026d0                MotorControl_Stop
 .text.MC_WClearFault
                0x00002708       0x28 ./MotorControl_App/MCFPGAIF.o
                0x00002708                MC_WClearFault
 .text.MC_GetStatus
                0x00002730       0x14 ./MotorControl_App/MCFPGAIF.o
                0x00002730                MC_GetStatus
 .text.MC_BLDCSetDirn
                0x00002744       0x18 ./MotorControl_App/MCFPGAIF.o
                0x00002744                MC_BLDCSetDirn
 .text.MC_BLDCGetSpdI
                0x0000275c       0x8c ./MotorControl_App/MCFPGAIF.o
                0x0000275c                MC_BLDCGetSpdI
 .text.MC_BLDCSetFabReg
                0x000027e8      0x214 ./MotorControl_App/MCFPGAIF.o
                0x000027e8                MC_BLDCSetFabReg
 .text.MC_StepperSetDirn
                0x000029fc       0x28 ./MotorControl_App/MCFPGAIF.o
                0x000029fc                MC_StepperSetDirn
 .text.MC_StepperGetI
                0x00002a24       0x34 ./MotorControl_App/MCFPGAIF.o
                0x00002a24                MC_StepperGetI
 .text.BLDC_SetSpeedSRamp
                0x00002a58       0x48 ./MotorControl_App/MCFPGAIF.o
                0x00002a58                BLDC_SetSpeedSRamp
 .text.MC_StepperSetFabReg
                0x00002aa0      0x140 ./MotorControl_App/MCFPGAIF.o
                0x00002aa0                MC_StepperSetFabReg
 .text.MotorControl_Init
                0x00002be0       0x1e ./MotorControl_App/MCFPGAIF.o
                0x00002be0                MotorControl_Init
 *fill*         0x00002bfe        0x2 
 .text.USB_init
                0x00002c00       0x70 ./MotorControl_App/USBMsgHandler.o
                0x00002c00                USB_init
 .text.USBMsgHandler
                0x00002c70      0x554 ./MotorControl_App/USBMsgHandler.o
                0x00002c70                USBMsgHandler
 .text.SendStreamDATA
                0x000031c4       0xc4 ./MotorControl_App/USBMsgHandler.o
                0x000031c4                SendStreamDATA
 .text.startup.main
                0x00003288       0xdc ./MotorControl_App/main.o
                0x00003288                main
 .text.hid_device_descriptor
                0x00003364        0xc ./MotorControl_App/usb_user_descriptors.o
 .text.hid_device_qual_descriptor
                0x00003370       0x18 ./MotorControl_App/usb_user_descriptors.o
 .text.hid_get_string.constprop.0
                0x00003388       0x34 ./MotorControl_App/usb_user_descriptors.o
 .text.hid_string_descriptor
                0x000033bc       0x5c ./MotorControl_App/usb_user_descriptors.o
 .text.__libc_init_array
                0x00003418       0x4c f:/microsemi/softconsole_v4.0/arm-none-eabi-gcc/bin/../lib/gcc/arm-none-eabi/4.9.3/../../../../arm-none-eabi/lib/armv7-m\libg_nano.a(lib_a-init.o)
                0x00003418                __libc_init_array
 *(.plt)
 *(.gnu.warning)
 *(.glue_7t)
 .glue_7t       0x00000000        0x0 linker stubs
 *(.glue_7)
 .glue_7        0x00000000        0x0 linker stubs
 *(.vfp11_veneer)
 .vfp11_veneer  0x00000000        0x0 linker stubs
                0x00003464                . = ALIGN (0x4)
 *crtbegin.o(.ctors)
 *(EXCLUDE_FILE(*crtend.o) .ctors)
 *(SORT(.ctors.*))
 *crtend.o(.ctors)
 *crtbegin.o(.dtors)
 *(EXCLUDE_FILE(*crtend.o) .dtors)
 *(SORT(.dtors.*))
 *crtend.o(.dtors)
 *(.rodata .rodata.* .gnu.linkonce.r.*)
 .rodata.CSWTCH.97
                0x00003464        0x6 ./MotorControl_Drivers/firmware/drivers/mss_usb/mss_usb_device.o
 .rodata.CSWTCH.95
                0x0000346a        0x6 ./MotorControl_Drivers/firmware/drivers/mss_usb/mss_usb_device.o
 .rodata.str1.1
                0x00003470       0x32 ./MotorControl_App/usb_user_descriptors.o
 *(.ARM.extab* .gnu.linkonce.armextab.*)
 *(.gcc_except_table)
 *(.eh_frame_hdr)
 *(.eh_frame)
 *fill*         0x000034a2        0x2 
 .eh_frame      0x000034a4        0x0 f:/microsemi/softconsole_v4.0/arm-none-eabi-gcc/bin/../lib/gcc/arm-none-eabi/4.9.3/armv7-m/crtbegin.o
 *(.vector_table)
 *(.init)
 .init          0x000034a4        0x4 f:/microsemi/softconsole_v4.0/arm-none-eabi-gcc/bin/../lib/gcc/arm-none-eabi/4.9.3/armv7-m/crti.o
                0x000034a4                _init
 .init          0x000034a8        0x8 f:/microsemi/softconsole_v4.0/arm-none-eabi-gcc/bin/../lib/gcc/arm-none-eabi/4.9.3/armv7-m/crtn.o
 *(.fini)
 .fini          0x000034b0        0x4 f:/microsemi/softconsole_v4.0/arm-none-eabi-gcc/bin/../lib/gcc/arm-none-eabi/4.9.3/armv7-m/crti.o
                0x000034b0                _fini
 .fini          0x000034b4        0x8 f:/microsemi/softconsole_v4.0/arm-none-eabi-gcc/bin/../lib/gcc/arm-none-eabi/4.9.3/armv7-m/crtn.o
                0x000034bc                PROVIDE (__preinit_array_start, .)
 *(.preinit_array)
                0x000034bc                PROVIDE (__preinit_array_end, .)
                0x000034bc                PROVIDE (__init_array_start, .)
 *(SORT(.init_array.*))
 *(.init_array)
 .init_array    0x000034bc        0x4 f:/microsemi/softconsole_v4.0/arm-none-eabi-gcc/bin/../lib/gcc/arm-none-eabi/4.9.3/armv7-m/crtbegin.o
                0x000034c0                PROVIDE (__init_array_end, .)
                0x000034c0                PROVIDE (__fini_array_start, .)
 *(.fini_array)
 .fini_array    0x000034c0        0x4 f:/microsemi/softconsole_v4.0/arm-none-eabi-gcc/bin/../lib/gcc/arm-none-eabi/4.9.3/armv7-m/crtbegin.o
 *(SORT(.fini_array.*))
                0x000034c4                PROVIDE (__fini_array_end, .)
                0x000034d0                . = ALIGN (0x10)
 *fill*         0x000034c4        0xc 
                0x000034d0                __exidx_start = .

.v4_bx          0x000034d0        0x0
 .v4_bx         0x00000000        0x0 linker stubs

.iplt           0x000034d0        0x0
 .iplt          0x00000000        0x0 f:/microsemi/softconsole_v4.0/arm-none-eabi-gcc/bin/../lib/gcc/arm-none-eabi/4.9.3/armv7-m/crtbegin.o

.rel.dyn        0x000034d0        0x0
 .rel.iplt      0x00000000        0x0 f:/microsemi/softconsole_v4.0/arm-none-eabi-gcc/bin/../lib/gcc/arm-none-eabi/4.9.3/armv7-m/crtbegin.o

.ARM.exidx
 *(.ARM.exidx* .gnu.linkonce.armexidx.*)
                0x000034d0                __exidx_end = .
                0x000034d0                _etext = .

.data           0x20000000       0xf0 load address 0x000034d0
                0x000034d0                __data_load = LOADADDR (.data)
                0x000034d0                _sidata = LOADADDR (.data)
                0x20000000                __data_start = .
                0x20000000                _sdata = .
 *(.jcr)
 .jcr           0x20000000        0x0 f:/microsemi/softconsole_v4.0/arm-none-eabi-gcc/bin/../lib/gcc/arm-none-eabi/4.9.3/armv7-m/crtbegin.o
 .jcr           0x20000000        0x4 f:/microsemi/softconsole_v4.0/arm-none-eabi-gcc/bin/../lib/gcc/arm-none-eabi/4.9.3/armv7-m/crtend.o
 *(.got.plt)
 *(.got)
 *(.shdata)
 *(.data .data.* .gnu.linkonce.d.*)
 .data.g_mss_usbd_cb
                0x20000004       0x28 ./MotorControl_Drivers/firmware/drivers/mss_usb/mss_usb_device.o
                0x20000004                g_mss_usbd_cb
 .data.usbd_hid_cb
                0x2000002c       0x20 ./MotorControl_Drivers/firmware/drivers/mss_usb/mss_usb_device_hid.o
                0x2000002c                usbd_hid_cb
 .data.hid_conf_descr
                0x2000004c       0x29 ./MotorControl_Drivers/firmware/drivers/mss_usb/mss_usb_device_hid.o
                0x2000004c                hid_conf_descr
 *fill*         0x20000075        0x3 
 .data.g_tx_complete_status
                0x20000078        0x4 ./MotorControl_Drivers/firmware/drivers/mss_usb/mss_usb_device_hid.o
                0x20000078                g_tx_complete_status
 .data.report_descr
                0x2000007c       0x34 ./MotorControl_Drivers/firmware/drivers/mss_usb/mss_usb_device_hid.o
                0x2000007c                report_descr
 .data.g_rx_complete_status
                0x200000b0        0x4 ./MotorControl_Drivers/firmware/drivers/mss_usb/mss_usb_device_hid.o
                0x200000b0                g_rx_complete_status
 .data.g_streamdata
                0x200000b4        0x1 ./MotorControl_App/USBMsgHandler.o
                0x200000b4                g_streamdata
 .data.g_streamaxis
                0x200000b5        0x1 ./MotorControl_App/USBMsgHandler.o
                0x200000b5                g_streamaxis
 .data.hs_dev_qualifier_descriptor.6847
                0x200000b6        0xa ./MotorControl_App/usb_user_descriptors.o
 .data.hid_mouse_descriptors_cb
                0x200000c0        0xc ./MotorControl_App/usb_user_descriptors.o
                0x200000c0                hid_mouse_descriptors_cb
 .data.fs_dev_qualifier_descriptor.6846
                0x200000cc        0xa ./MotorControl_App/usb_user_descriptors.o
 .data.device_descriptor.6841
                0x200000d6       0x12 ./MotorControl_App/usb_user_descriptors.o
 .data.lang_string_descriptor.6854
                0x200000e8        0x4 ./MotorControl_App/usb_user_descriptors.o
                0x200000f0                . = ALIGN (0x10)
 *fill*         0x200000ec        0x4 
                0x200000f0                _edata = .

.igot.plt       0x200000f0        0x0 load address 0x000035c0
 .igot.plt      0x00000000        0x0 f:/microsemi/softconsole_v4.0/arm-none-eabi-gcc/bin/../lib/gcc/arm-none-eabi/4.9.3/armv7-m/crtbegin.o

.bss            0x200000f0      0x3e0 load address 0x000035c0
                0x200000f0                __bss_start__ = .
                0x200000f0                _sbss = .
 *(.shbss)
 *(.bss .bss.* .gnu.linkonce.b.*)
 .bss           0x200000f0       0x1c f:/microsemi/softconsole_v4.0/arm-none-eabi-gcc/bin/../lib/gcc/arm-none-eabi/4.9.3/armv7-m/crtbegin.o
 .bss.g_usbd_user_speed
                0x2000010c        0x1 ./MotorControl_Drivers/firmware/drivers/mss_usb/mss_usb_device.o
 *fill*         0x2000010d        0x1 
 .bss.g_setup_pkt
                0x2000010e        0x8 ./MotorControl_Drivers/firmware/drivers/mss_usb/mss_usb_device.o
 *fill*         0x20000116        0x2 
 .bss.device_rx_ep
                0x20000118       0xdc ./MotorControl_Drivers/firmware/drivers/mss_usb/mss_usb_device.o
 .bss.g_usbd_dev_conf
                0x200001f4        0xe ./MotorControl_Drivers/firmware/drivers/mss_usb/mss_usb_device.o
 *fill*         0x20000202        0x2 
 .bss.device_tx_ep
                0x20000204       0xdc ./MotorControl_Drivers/firmware/drivers/mss_usb/mss_usb_device.o
 .bss.g_usbd_status
                0x200002e0        0x2 ./MotorControl_Drivers/firmware/drivers/mss_usb/mss_usb_device.o
 .bss.g_rx_data
                0x200002e2       0x19 ./MotorControl_Drivers/firmware/drivers/mss_usb/mss_usb_device_hid.o
                0x200002e2                g_rx_data
 .bss.g_hid_state
                0x200002fb        0x1 ./MotorControl_Drivers/firmware/drivers/mss_usb/mss_usb_device_hid.o
                0x200002fb                g_hid_state
 .bss.g_comblk_response_size
                0x200002fc        0x2 ./MotorControl_Drivers/firmware/drivers/mss_sys_services/mss_comblk.o
 *fill*         0x200002fe        0x2 
 .bss.g_comblk_page_handler
                0x20000300        0x4 ./MotorControl_Drivers/firmware/drivers/mss_sys_services/mss_comblk.o
 .bss.g_comblk_p_cmd
                0x20000304        0x4 ./MotorControl_Drivers/firmware/drivers/mss_sys_services/mss_comblk.o
 .bss.g_request_in_progress
                0x20000308        0x1 ./MotorControl_Drivers/firmware/drivers/mss_sys_services/mss_comblk.o
 *fill*         0x20000309        0x3 
 .bss.g_async_event_handler
                0x2000030c        0x4 ./MotorControl_Drivers/firmware/drivers/mss_sys_services/mss_comblk.o
 .bss.g_comblk_cmd_size
                0x20000310        0x2 ./MotorControl_Drivers/firmware/drivers/mss_sys_services/mss_comblk.o
 *fill*         0x20000312        0x2 
 .bss.g_comblk_p_data
                0x20000314        0x4 ./MotorControl_Drivers/firmware/drivers/mss_sys_services/mss_comblk.o
 .bss.g_comblk_completion_handler
                0x20000318        0x4 ./MotorControl_Drivers/firmware/drivers/mss_sys_services/mss_comblk.o
 .bss.g_comblk_response_idx
                0x2000031c        0x2 ./MotorControl_Drivers/firmware/drivers/mss_sys_services/mss_comblk.o
 *fill*         0x2000031e        0x2 
 .bss.g_comblk_data_size
                0x20000320        0x4 ./MotorControl_Drivers/firmware/drivers/mss_sys_services/mss_comblk.o
 .bss.g_comblk_p_response
                0x20000324        0x4 ./MotorControl_Drivers/firmware/drivers/mss_sys_services/mss_comblk.o
 .bss.g_comblk_state
                0x20000328        0x1 ./MotorControl_Drivers/firmware/drivers/mss_sys_services/mss_comblk.o
 .bss.g_comblk_cmd_opcode
                0x20000329        0x1 ./MotorControl_Drivers/firmware/drivers/mss_sys_services/mss_comblk.o
 *fill*         0x2000032a        0x2 
 .bss.g_transfer
                0x2000032c       0x18 ./MotorControl_Drivers/firmware/drivers/mss_hpdma/mss_hpdma.o
 .bss.g_report  0x20000344       0x19 ./MotorControl_App/USBMsgHandler.o
 .bss.g_string_descriptor.6855
                0x2000035d       0x40 ./MotorControl_App/usb_user_descriptors.o
 *(COMMON)
 *fill*         0x2000039d        0x3 
 COMMON         0x200003a0        0x8 ./MotorControl_Drivers/firmware/drivers/mss_usb/mss_usb_device.o
                0x200003a0                g_usbd_class_cb
                0x200003a4                g_usbd_user_descr_cb
 COMMON         0x200003a8       0x2c ./MotorControl_Drivers/firmware/drivers/mss_usb/mss_usb_device_cif.o
                0x200003a8                gd_tx_ep
                0x200003bc                cep_state
                0x200003c0                gd_rx_ep
 COMMON         0x200003d4        0x1 ./MotorControl_Drivers/firmware/drivers/mss_usb/mss_usb_device_hid.o
                0x200003d4                g_usbd_hid_user_speed
 *fill*         0x200003d5        0x3 
 COMMON         0x200003d8       0xe8 ./MotorControl_App/MCCalc.o
                0x200003d8                g_hall_sensor_pol
                0x200003dc                g_LX_PWM_freq_kHz
                0x200003e0                g_theta_factor
                0x200003e4                g_pwm_period_st
                0x200003e8                g_en_angle_cnt_max
                0x200003ec                g_slew_count_st
                0x200003f0                g_en_speed_window
                0x200003f4                g_speed_scale
                0x200003f8                g_pwm_period
                0x200003fc                g_slew_count
                0x20000400                g_rate_count
                0x20000404                g_en_speed_factor
                0x20000408                g_rate_count_st
                0x2000040c                g_bldc1
                0x20000424                g_pwm_gain
                0x20000428                g_adc_scale_st
                0x2000042c                g_algorithm
                0x20000430                g_stepper
                0x20000468                g_adc_scale
                0x2000046c                g_mc_bldc_foc
                0x200004b8                g_speed_descale
                0x200004bc                g_en_angle_factor
 COMMON         0x200004c0        0xc ./MotorControl_App/MCFPGAIF.o
                0x200004c0                speedbuf
                0x200004c4                g_base_addr
                0x200004c8                currentbuf
                0x200004d0                . = ALIGN (0x10)
 *fill*         0x200004cc        0x4 
                0x200004d0                __bss_end__ = .
                0x200004d0                _end = .
                0x200004d0                __end = _end
                0x200004d0                _ebss = .
                0x200004d0                PROVIDE (end, .)

.heap           0x200004d0     0xeb30 load address 0x000035c0
                0x200004d0                __heap_start__ = .
                0x200014d0                . = (. + MIN_SIZE_HEAP)
 *fill*         0x200004d0     0x1000 
                0x2000f000                . = (. + (((ABSOLUTE (RAM_START_ADDRESS) + RAM_SIZE) - MAIN_STACK_SIZE) - .))
 *fill*         0x200014d0     0xdb30 
                0x2000f000                _eheap = .

.stack          0x2000f000     0x1000 load address 0x000035c0
                0x2000f000                __stack_start__ = .
                0x20010000                . = (. + MAIN_STACK_SIZE)
 *fill*         0x2000f000     0x1000 
                0x20010000                _estack = .

.stab
 *(.stab)

.stabstr
 *(.stabstr)

.debug
 *(.debug)

.line
 *(.line)

.debug_srcinfo
 *(.debug_srcinfo)

.debug_sfnames
 *(.debug_sfnames)

.debug_aranges  0x00000000      0xab8
 *(.debug_aranges)
 .debug_aranges
                0x00000000       0x20 ./MotorControl_Drivers/firmware/hal/CortexM3/GNU/hal.o
 .debug_aranges
                0x00000020       0x20 ./MotorControl_Drivers/firmware/hal/CortexM3/GNU/hw_reg_access.o
 .debug_aranges
                0x00000040       0x48 ./MotorControl_Drivers/firmware/hal/CortexM3/cortex_nvic.o
 .debug_aranges
                0x00000088       0x18 ./MotorControl_Drivers/firmware/drivers_config/sys_config/sys_config.o
 .debug_aranges
                0x000000a0       0x58 ./MotorControl_Drivers/firmware/drivers/mss_usb/mss_usb_common_cif.o
 .debug_aranges
                0x000000f8      0x168 ./MotorControl_Drivers/firmware/drivers/mss_usb/mss_usb_device.o
 .debug_aranges
                0x00000260       0x78 ./MotorControl_Drivers/firmware/drivers/mss_usb/mss_usb_device_cdc.o
 .debug_aranges
                0x000002d8       0x60 ./MotorControl_Drivers/firmware/drivers/mss_usb/mss_usb_device_cif.o
 .debug_aranges
                0x00000338       0x80 ./MotorControl_Drivers/firmware/drivers/mss_usb/mss_usb_device_hid.o
 .debug_aranges
                0x000003b8       0xa0 ./MotorControl_Drivers/firmware/drivers/mss_usb/mss_usb_device_msd.o
 .debug_aranges
                0x00000458       0x80 ./MotorControl_Drivers/firmware/drivers/mss_usb/mss_usb_device_printer.o
 .debug_aranges
                0x000004d8       0x60 ./MotorControl_Drivers/firmware/drivers/mss_usb/mss_usb_device_vendor.o
 .debug_aranges
                0x00000538       0x18 ./MotorControl_Drivers/firmware/drivers/mss_usb/mss_usb_host.o
 .debug_aranges
                0x00000550       0x18 ./MotorControl_Drivers/firmware/drivers/mss_usb/mss_usb_host_cif.o
 .debug_aranges
                0x00000568       0x18 ./MotorControl_Drivers/firmware/drivers/mss_usb/mss_usb_host_msc.o
 .debug_aranges
                0x00000580       0x68 ./MotorControl_Drivers/firmware/drivers/mss_sys_services/mss_comblk.o
 .debug_aranges
                0x000005e8      0x1a8 ./MotorControl_Drivers/firmware/drivers/mss_sys_services/mss_sys_services.o
 .debug_aranges
                0x00000790       0x48 ./MotorControl_Drivers/firmware/drivers/mss_nvm/mss_nvm.o
 .debug_aranges
                0x000007d8       0x60 ./MotorControl_Drivers/firmware/drivers/mss_hpdma/mss_hpdma.o
 .debug_aranges
                0x00000838       0x50 ./MotorControl_Drivers/firmware/drivers/mss_gpio/mss_gpio.o
 .debug_aranges
                0x00000888       0xa8 ./MotorControl_Drivers/firmware/CMSIS/startup_gcc/newlib_stubs.o
 .debug_aranges
                0x00000930       0x20 ./MotorControl_Drivers/firmware/CMSIS/startup_gcc/startup_m2sxxx.o
 .debug_aranges
                0x00000950       0x30 ./MotorControl_Drivers/firmware/CMSIS/system_m2sxxx.o
 .debug_aranges
                0x00000980       0x38 ./MotorControl_App/MCCalc.o
 .debug_aranges
                0x000009b8       0x78 ./MotorControl_App/MCFPGAIF.o
 .debug_aranges
                0x00000a30       0x30 ./MotorControl_App/USBMsgHandler.o
 .debug_aranges
                0x00000a60       0x20 ./MotorControl_App/main.o
 .debug_aranges
                0x00000a80       0x38 ./MotorControl_App/usb_user_descriptors.o

.debug_pubnames
 *(.debug_pubnames)

.debug_info     0x00000000    0x14d1c
 *(.debug_info .gnu.linkonce.wi.*)
 .debug_info    0x00000000       0xae ./MotorControl_Drivers/firmware/hal/CortexM3/GNU/hal.o
 .debug_info    0x000000ae       0xb8 ./MotorControl_Drivers/firmware/hal/CortexM3/GNU/hw_reg_access.o
 .debug_info    0x00000166      0x180 ./MotorControl_Drivers/firmware/hal/CortexM3/cortex_nvic.o
 .debug_info    0x000002e6       0x92 ./MotorControl_Drivers/firmware/drivers_config/sys_config/sys_config.o
 .debug_info    0x00000378     0x2875 ./MotorControl_Drivers/firmware/drivers/mss_usb/mss_usb_common_cif.o
 .debug_info    0x00002bed     0x247b ./MotorControl_Drivers/firmware/drivers/mss_usb/mss_usb_device.o
 .debug_info    0x00005068      0xa4f ./MotorControl_Drivers/firmware/drivers/mss_usb/mss_usb_device_cdc.o
 .debug_info    0x00005ab7     0x19e9 ./MotorControl_Drivers/firmware/drivers/mss_usb/mss_usb_device_cif.o
 .debug_info    0x000074a0      0x8ea ./MotorControl_Drivers/firmware/drivers/mss_usb/mss_usb_device_hid.o
 .debug_info    0x00007d8a     0x1384 ./MotorControl_Drivers/firmware/drivers/mss_usb/mss_usb_device_msd.o
 .debug_info    0x0000910e      0x995 ./MotorControl_Drivers/firmware/drivers/mss_usb/mss_usb_device_printer.o
 .debug_info    0x00009aa3      0x96d ./MotorControl_Drivers/firmware/drivers/mss_usb/mss_usb_device_vendor.o
 .debug_info    0x0000a410       0xa0 ./MotorControl_Drivers/firmware/drivers/mss_usb/mss_usb_host.o
 .debug_info    0x0000a4b0       0x92 ./MotorControl_Drivers/firmware/drivers/mss_usb/mss_usb_host_cif.o
 .debug_info    0x0000a542       0xa0 ./MotorControl_Drivers/firmware/drivers/mss_usb/mss_usb_host_msc.o
 .debug_info    0x0000a5e2      0xd97 ./MotorControl_Drivers/firmware/drivers/mss_sys_services/mss_comblk.o
 .debug_info    0x0000b379     0x281c ./MotorControl_Drivers/firmware/drivers/mss_sys_services/mss_sys_services.o
 .debug_info    0x0000db95     0x122b ./MotorControl_Drivers/firmware/drivers/mss_nvm/mss_nvm.o
 .debug_info    0x0000edc0     0x110a ./MotorControl_Drivers/firmware/drivers/mss_hpdma/mss_hpdma.o
 .debug_info    0x0000feca     0x103f ./MotorControl_Drivers/firmware/drivers/mss_gpio/mss_gpio.o
 .debug_info    0x00010f09      0x707 ./MotorControl_Drivers/firmware/CMSIS/startup_gcc/newlib_stubs.o
 .debug_info    0x00011610       0xba ./MotorControl_Drivers/firmware/CMSIS/startup_gcc/startup_m2sxxx.o
 .debug_info    0x000116ca      0xb11 ./MotorControl_Drivers/firmware/CMSIS/system_m2sxxx.o
 .debug_info    0x000121db      0x5ba ./MotorControl_App/MCCalc.o
 .debug_info    0x00012795      0xace ./MotorControl_App/MCFPGAIF.o
 .debug_info    0x00013263     0x132b ./MotorControl_App/USBMsgHandler.o
 .debug_info    0x0001458e      0x416 ./MotorControl_App/main.o
 .debug_info    0x000149a4      0x378 ./MotorControl_App/usb_user_descriptors.o

.debug_abbrev   0x00000000     0x352a
 *(.debug_abbrev)
 .debug_abbrev  0x00000000       0x14 ./MotorControl_Drivers/firmware/hal/CortexM3/GNU/hal.o
 .debug_abbrev  0x00000014       0x14 ./MotorControl_Drivers/firmware/hal/CortexM3/GNU/hw_reg_access.o
 .debug_abbrev  0x00000028       0xa0 ./MotorControl_Drivers/firmware/hal/CortexM3/cortex_nvic.o
 .debug_abbrev  0x000000c8       0x4b ./MotorControl_Drivers/firmware/drivers_config/sys_config/sys_config.o
 .debug_abbrev  0x00000113      0x427 ./MotorControl_Drivers/firmware/drivers/mss_usb/mss_usb_common_cif.o
 .debug_abbrev  0x0000053a      0x504 ./MotorControl_Drivers/firmware/drivers/mss_usb/mss_usb_device.o
 .debug_abbrev  0x00000a3e      0x2f3 ./MotorControl_Drivers/firmware/drivers/mss_usb/mss_usb_device_cdc.o
 .debug_abbrev  0x00000d31      0x356 ./MotorControl_Drivers/firmware/drivers/mss_usb/mss_usb_device_cif.o
 .debug_abbrev  0x00001087      0x280 ./MotorControl_Drivers/firmware/drivers/mss_usb/mss_usb_device_hid.o
 .debug_abbrev  0x00001307      0x303 ./MotorControl_Drivers/firmware/drivers/mss_usb/mss_usb_device_msd.o
 .debug_abbrev  0x0000160a      0x263 ./MotorControl_Drivers/firmware/drivers/mss_usb/mss_usb_device_printer.o
 .debug_abbrev  0x0000186d      0x226 ./MotorControl_Drivers/firmware/drivers/mss_usb/mss_usb_device_vendor.o
 .debug_abbrev  0x00001a93       0x4b ./MotorControl_Drivers/firmware/drivers/mss_usb/mss_usb_host.o
 .debug_abbrev  0x00001ade       0x4b ./MotorControl_Drivers/firmware/drivers/mss_usb/mss_usb_host_cif.o
 .debug_abbrev  0x00001b29       0x4b ./MotorControl_Drivers/firmware/drivers/mss_usb/mss_usb_host_msc.o
 .debug_abbrev  0x00001b74      0x316 ./MotorControl_Drivers/firmware/drivers/mss_sys_services/mss_comblk.o
 .debug_abbrev  0x00001e8a      0x2d6 ./MotorControl_Drivers/firmware/drivers/mss_sys_services/mss_sys_services.o
 .debug_abbrev  0x00002160      0x32b ./MotorControl_Drivers/firmware/drivers/mss_nvm/mss_nvm.o
 .debug_abbrev  0x0000248b      0x24f ./MotorControl_Drivers/firmware/drivers/mss_hpdma/mss_hpdma.o
 .debug_abbrev  0x000026da      0x1e8 ./MotorControl_Drivers/firmware/drivers/mss_gpio/mss_gpio.o
 .debug_abbrev  0x000028c2      0x222 ./MotorControl_Drivers/firmware/CMSIS/startup_gcc/newlib_stubs.o
 .debug_abbrev  0x00002ae4       0x14 ./MotorControl_Drivers/firmware/CMSIS/startup_gcc/startup_m2sxxx.o
 .debug_abbrev  0x00002af8      0x1ee ./MotorControl_Drivers/firmware/CMSIS/system_m2sxxx.o
 .debug_abbrev  0x00002ce6       0xdd ./MotorControl_App/MCCalc.o
 .debug_abbrev  0x00002dc3      0x223 ./MotorControl_App/MCFPGAIF.o
 .debug_abbrev  0x00002fe6      0x2bc ./MotorControl_App/USBMsgHandler.o
 .debug_abbrev  0x000032a2       0xf8 ./MotorControl_App/main.o
 .debug_abbrev  0x0000339a      0x190 ./MotorControl_App/usb_user_descriptors.o

.debug_line     0x00000000     0x5ac7
 *(.debug_line)
 .debug_line    0x00000000       0x6b ./MotorControl_Drivers/firmware/hal/CortexM3/GNU/hal.o
 .debug_line    0x0000006b       0xa9 ./MotorControl_Drivers/firmware/hal/CortexM3/GNU/hw_reg_access.o
 .debug_line    0x00000114      0x194 ./MotorControl_Drivers/firmware/hal/CortexM3/cortex_nvic.o
 .debug_line    0x000002a8      0x115 ./MotorControl_Drivers/firmware/drivers_config/sys_config/sys_config.o
 .debug_line    0x000003bd      0x742 ./MotorControl_Drivers/firmware/drivers/mss_usb/mss_usb_common_cif.o
 .debug_line    0x00000aff      0x8fe ./MotorControl_Drivers/firmware/drivers/mss_usb/mss_usb_device.o
 .debug_line    0x000013fd      0x2b1 ./MotorControl_Drivers/firmware/drivers/mss_usb/mss_usb_device_cdc.o
 .debug_line    0x000016ae      0x42c ./MotorControl_Drivers/firmware/drivers/mss_usb/mss_usb_device_cif.o
 .debug_line    0x00001ada      0x2ba ./MotorControl_Drivers/firmware/drivers/mss_usb/mss_usb_device_hid.o
 .debug_line    0x00001d94      0x549 ./MotorControl_Drivers/firmware/drivers/mss_usb/mss_usb_device_msd.o
 .debug_line    0x000022dd      0x2c4 ./MotorControl_Drivers/firmware/drivers/mss_usb/mss_usb_device_printer.o
 .debug_line    0x000025a1      0x2b7 ./MotorControl_Drivers/firmware/drivers/mss_usb/mss_usb_device_vendor.o
 .debug_line    0x00002858      0x115 ./MotorControl_Drivers/firmware/drivers/mss_usb/mss_usb_host.o
 .debug_line    0x0000296d      0x115 ./MotorControl_Drivers/firmware/drivers/mss_usb/mss_usb_host_cif.o
 .debug_line    0x00002a82      0x115 ./MotorControl_Drivers/firmware/drivers/mss_usb/mss_usb_host_msc.o
 .debug_line    0x00002b97      0x484 ./MotorControl_Drivers/firmware/drivers/mss_sys_services/mss_comblk.o
 .debug_line    0x0000301b      0xaea ./MotorControl_Drivers/firmware/drivers/mss_sys_services/mss_sys_services.o
 .debug_line    0x00003b05      0x391 ./MotorControl_Drivers/firmware/drivers/mss_nvm/mss_nvm.o
 .debug_line    0x00003e96      0x2c9 ./MotorControl_Drivers/firmware/drivers/mss_hpdma/mss_hpdma.o
 .debug_line    0x0000415f      0x2d7 ./MotorControl_Drivers/firmware/drivers/mss_gpio/mss_gpio.o
 .debug_line    0x00004436      0x23d ./MotorControl_Drivers/firmware/CMSIS/startup_gcc/newlib_stubs.o
 .debug_line    0x00004673      0x1ae ./MotorControl_Drivers/firmware/CMSIS/startup_gcc/startup_m2sxxx.o
 .debug_line    0x00004821      0x1d6 ./MotorControl_Drivers/firmware/CMSIS/system_m2sxxx.o
 .debug_line    0x000049f7      0x1ff ./MotorControl_App/MCCalc.o
 .debug_line    0x00004bf6      0x3c7 ./MotorControl_App/MCFPGAIF.o
 .debug_line    0x00004fbd      0x616 ./MotorControl_App/USBMsgHandler.o
 .debug_line    0x000055d3      0x2aa ./MotorControl_App/main.o
 .debug_line    0x0000587d      0x24a ./MotorControl_App/usb_user_descriptors.o

.debug_frame    0x00000000     0x1a68
 *(.debug_frame)
 .debug_frame   0x00000000       0x70 ./MotorControl_Drivers/firmware/hal/CortexM3/cortex_nvic.o
 .debug_frame   0x00000070      0x128 ./MotorControl_Drivers/firmware/drivers/mss_usb/mss_usb_common_cif.o
 .debug_frame   0x00000198      0x3b8 ./MotorControl_Drivers/firmware/drivers/mss_usb/mss_usb_device.o
 .debug_frame   0x00000550      0x120 ./MotorControl_Drivers/firmware/drivers/mss_usb/mss_usb_device_cdc.o
 .debug_frame   0x00000670       0xcc ./MotorControl_Drivers/firmware/drivers/mss_usb/mss_usb_device_cif.o
 .debug_frame   0x0000073c      0x110 ./MotorControl_Drivers/firmware/drivers/mss_usb/mss_usb_device_hid.o
 .debug_frame   0x0000084c      0x1b8 ./MotorControl_Drivers/firmware/drivers/mss_usb/mss_usb_device_msd.o
 .debug_frame   0x00000a04      0x124 ./MotorControl_Drivers/firmware/drivers/mss_usb/mss_usb_device_printer.o
 .debug_frame   0x00000b28       0xd4 ./MotorControl_Drivers/firmware/drivers/mss_usb/mss_usb_device_vendor.o
 .debug_frame   0x00000bfc      0x13c ./MotorControl_Drivers/firmware/drivers/mss_sys_services/mss_comblk.o
 .debug_frame   0x00000d38      0x56c ./MotorControl_Drivers/firmware/drivers/mss_sys_services/mss_sys_services.o
 .debug_frame   0x000012a4       0xcc ./MotorControl_Drivers/firmware/drivers/mss_nvm/mss_nvm.o
 .debug_frame   0x00001370       0xd4 ./MotorControl_Drivers/firmware/drivers/mss_hpdma/mss_hpdma.o
 .debug_frame   0x00001444       0x88 ./MotorControl_Drivers/firmware/drivers/mss_gpio/mss_gpio.o
 .debug_frame   0x000014cc      0x160 ./MotorControl_Drivers/firmware/CMSIS/startup_gcc/newlib_stubs.o
 .debug_frame   0x0000162c       0x4c ./MotorControl_Drivers/firmware/CMSIS/system_m2sxxx.o
 .debug_frame   0x00001678       0x6c ./MotorControl_App/MCCalc.o
 .debug_frame   0x000016e4      0x154 ./MotorControl_App/MCFPGAIF.o
 .debug_frame   0x00001838       0xe8 ./MotorControl_App/USBMsgHandler.o
 .debug_frame   0x00001920       0x28 ./MotorControl_App/main.o
 .debug_frame   0x00001948       0x64 ./MotorControl_App/usb_user_descriptors.o
 .debug_frame   0x000019ac       0x20 f:/microsemi/softconsole_v4.0/arm-none-eabi-gcc/bin/../lib/gcc/arm-none-eabi/4.9.3/../../../../arm-none-eabi/lib/armv7-m\libg_nano.a(lib_a-errno.o)
 .debug_frame   0x000019cc       0x28 f:/microsemi/softconsole_v4.0/arm-none-eabi-gcc/bin/../lib/gcc/arm-none-eabi/4.9.3/../../../../arm-none-eabi/lib/armv7-m\libg_nano.a(lib_a-exit.o)
 .debug_frame   0x000019f4       0x2c f:/microsemi/softconsole_v4.0/arm-none-eabi-gcc/bin/../lib/gcc/arm-none-eabi/4.9.3/../../../../arm-none-eabi/lib/armv7-m\libg_nano.a(lib_a-init.o)
 .debug_frame   0x00001a20       0x28 f:/microsemi/softconsole_v4.0/arm-none-eabi-gcc/bin/../lib/gcc/arm-none-eabi/4.9.3/../../../../arm-none-eabi/lib/armv7-m\libg_nano.a(lib_a-memcpy.o)
 .debug_frame   0x00001a48       0x20 f:/microsemi/softconsole_v4.0/arm-none-eabi-gcc/bin/../lib/gcc/arm-none-eabi/4.9.3/../../../../arm-none-eabi/lib/armv7-m\libg_nano.a(lib_a-memset.o)

.debug_str      0x00000000     0x6a53
 *(.debug_str)
 .debug_str     0x00000000      0x24d ./MotorControl_Drivers/firmware/hal/CortexM3/cortex_nvic.o
                                0x29a (size before relaxing)
 .debug_str     0x0000024d       0x68 ./MotorControl_Drivers/firmware/drivers_config/sys_config/sys_config.o
                                0x1fa (size before relaxing)
 .debug_str     0x000002b5     0x17fe ./MotorControl_Drivers/firmware/drivers/mss_usb/mss_usb_common_cif.o
                               0x1ab8 (size before relaxing)
 .debug_str     0x00001ab3      0xdf0 ./MotorControl_Drivers/firmware/drivers/mss_usb/mss_usb_device.o
                               0x1900 (size before relaxing)
 .debug_str     0x000028a3      0x2df ./MotorControl_Drivers/firmware/drivers/mss_usb/mss_usb_device_cdc.o
                                0x86f (size before relaxing)
 .debug_str     0x00002b82      0x25e ./MotorControl_Drivers/firmware/drivers/mss_usb/mss_usb_device_cif.o
                               0x15a9 (size before relaxing)
 .debug_str     0x00002de0      0x242 ./MotorControl_Drivers/firmware/drivers/mss_usb/mss_usb_device_hid.o
                                0x80b (size before relaxing)
 .debug_str     0x00003022      0x800 ./MotorControl_Drivers/firmware/drivers/mss_usb/mss_usb_device_msd.o
                                0xe35 (size before relaxing)
 .debug_str     0x00003822      0x3cf ./MotorControl_Drivers/firmware/drivers/mss_usb/mss_usb_device_printer.o
                                0x9f9 (size before relaxing)
 .debug_str     0x00003bf1      0x1da ./MotorControl_Drivers/firmware/drivers/mss_usb/mss_usb_device_vendor.o
                                0x808 (size before relaxing)
 .debug_str     0x00003dcb       0x4c ./MotorControl_Drivers/firmware/drivers/mss_usb/mss_usb_host.o
                                0x203 (size before relaxing)
 .debug_str     0x00003e17       0x44 ./MotorControl_Drivers/firmware/drivers/mss_usb/mss_usb_host_cif.o
                                0x1f6 (size before relaxing)
 .debug_str     0x00003e5b       0x44 ./MotorControl_Drivers/firmware/drivers/mss_usb/mss_usb_host_msc.o
                                0x207 (size before relaxing)
 .debug_str     0x00003e9f      0x34f ./MotorControl_Drivers/firmware/drivers/mss_sys_services/mss_comblk.o
                                0xb6a (size before relaxing)
 .debug_str     0x000041ee     0x1050 ./MotorControl_Drivers/firmware/drivers/mss_sys_services/mss_sys_services.o
                               0x13ea (size before relaxing)
 .debug_str     0x0000523e      0x380 ./MotorControl_Drivers/firmware/drivers/mss_nvm/mss_nvm.o
                                0xccb (size before relaxing)
 .debug_str     0x000055be      0x4d7 ./MotorControl_Drivers/firmware/drivers/mss_hpdma/mss_hpdma.o
                               0x136e (size before relaxing)
 .debug_str     0x00005a95      0x49d ./MotorControl_Drivers/firmware/drivers/mss_gpio/mss_gpio.o
                               0x1319 (size before relaxing)
 .debug_str     0x00005f32      0x20d ./MotorControl_Drivers/firmware/CMSIS/startup_gcc/newlib_stubs.o
                                0x408 (size before relaxing)
 .debug_str     0x0000613f      0x21e ./MotorControl_Drivers/firmware/CMSIS/system_m2sxxx.o
                                0xb21 (size before relaxing)
 .debug_str     0x0000635d      0x3e8 ./MotorControl_App/MCCalc.o
                                0x5f0 (size before relaxing)
 .debug_str     0x00006745      0x151 ./MotorControl_App/MCFPGAIF.o
                                0x6fb (size before relaxing)
 .debug_str     0x00006896       0xbe ./MotorControl_App/USBMsgHandler.o
                                0xf02 (size before relaxing)
 .debug_str     0x00006954       0x20 ./MotorControl_App/main.o
                                0x466 (size before relaxing)
 .debug_str     0x00006974       0xdf ./MotorControl_App/usb_user_descriptors.o
                                0x3d9 (size before relaxing)

.debug_loc      0x00000000     0x6848
 *(.debug_loc)
 .debug_loc     0x00000000      0xe7a ./MotorControl_Drivers/firmware/drivers/mss_usb/mss_usb_common_cif.o
 .debug_loc     0x00000e7a      0xce5 ./MotorControl_Drivers/firmware/drivers/mss_usb/mss_usb_device.o
 .debug_loc     0x00001b5f      0x424 ./MotorControl_Drivers/firmware/drivers/mss_usb/mss_usb_device_cdc.o
 .debug_loc     0x00001f83      0x273 ./MotorControl_Drivers/firmware/drivers/mss_usb/mss_usb_device_cif.o
 .debug_loc     0x000021f6      0x413 ./MotorControl_Drivers/firmware/drivers/mss_usb/mss_usb_device_hid.o
 .debug_loc     0x00002609      0xc3d ./MotorControl_Drivers/firmware/drivers/mss_usb/mss_usb_device_msd.o
 .debug_loc     0x00003246      0x40a ./MotorControl_Drivers/firmware/drivers/mss_usb/mss_usb_device_printer.o
 .debug_loc     0x00003650      0x4c1 ./MotorControl_Drivers/firmware/drivers/mss_usb/mss_usb_device_vendor.o
 .debug_loc     0x00003b11      0x5ca ./MotorControl_Drivers/firmware/drivers/mss_sys_services/mss_comblk.o
 .debug_loc     0x000040db      0xf49 ./MotorControl_Drivers/firmware/drivers/mss_sys_services/mss_sys_services.o
 .debug_loc     0x00005024      0xd38 ./MotorControl_Drivers/firmware/drivers/mss_nvm/mss_nvm.o
 .debug_loc     0x00005d5c       0xae ./MotorControl_Drivers/firmware/drivers/mss_hpdma/mss_hpdma.o
 .debug_loc     0x00005e0a      0x1bc ./MotorControl_Drivers/firmware/drivers/mss_gpio/mss_gpio.o
 .debug_loc     0x00005fc6      0x291 ./MotorControl_Drivers/firmware/CMSIS/startup_gcc/newlib_stubs.o
 .debug_loc     0x00006257       0xb2 ./MotorControl_Drivers/firmware/CMSIS/system_m2sxxx.o
 .debug_loc     0x00006309      0x148 ./MotorControl_App/MCCalc.o
 .debug_loc     0x00006451      0x180 ./MotorControl_App/MCFPGAIF.o
 .debug_loc     0x000065d1      0x277 ./MotorControl_App/usb_user_descriptors.o

.debug_macinfo
 *(.debug_macinfo)

.debug_weaknames
 *(.debug_weaknames)

.debug_funcnames
 *(.debug_funcnames)

.debug_typenames
 *(.debug_typenames)

.debug_varnames
 *(.debug_varnames)

.note.gnu.arm.ident
 *(.note.gnu.arm.ident)

.ARM.attributes
                0x00000000       0x29
 *(.ARM.attributes)
 .ARM.attributes
                0x00000000       0x1d f:/microsemi/softconsole_v4.0/arm-none-eabi-gcc/bin/../lib/gcc/arm-none-eabi/4.9.3/armv7-m/crti.o
 .ARM.attributes
                0x0000001d       0x2d f:/microsemi/softconsole_v4.0/arm-none-eabi-gcc/bin/../lib/gcc/arm-none-eabi/4.9.3/armv7-m/crtbegin.o
 .ARM.attributes
                0x0000004a       0x1b f:/microsemi/softconsole_v4.0/arm-none-eabi-gcc/bin/../lib/gcc/arm-none-eabi/4.9.3/../../../../arm-none-eabi/lib/armv7-m/crt0.o
 .ARM.attributes
                0x00000065       0x21 ./MotorControl_Drivers/firmware/hal/CortexM3/GNU/hal.o
 .ARM.attributes
                0x00000086       0x21 ./MotorControl_Drivers/firmware/hal/CortexM3/GNU/hw_reg_access.o
 .ARM.attributes
                0x000000a7       0x33 ./MotorControl_Drivers/firmware/hal/CortexM3/cortex_nvic.o
 .ARM.attributes
                0x000000da       0x33 ./MotorControl_Drivers/firmware/drivers_config/sys_config/sys_config.o
 .ARM.attributes
                0x0000010d       0x33 ./MotorControl_Drivers/firmware/drivers/mss_usb/mss_usb_common_cif.o
 .ARM.attributes
                0x00000140       0x33 ./MotorControl_Drivers/firmware/drivers/mss_usb/mss_usb_device.o
 .ARM.attributes
                0x00000173       0x33 ./MotorControl_Drivers/firmware/drivers/mss_usb/mss_usb_device_cdc.o
 .ARM.attributes
                0x000001a6       0x33 ./MotorControl_Drivers/firmware/drivers/mss_usb/mss_usb_device_cif.o
 .ARM.attributes
                0x000001d9       0x33 ./MotorControl_Drivers/firmware/drivers/mss_usb/mss_usb_device_hid.o
 .ARM.attributes
                0x0000020c       0x33 ./MotorControl_Drivers/firmware/drivers/mss_usb/mss_usb_device_msd.o
 .ARM.attributes
                0x0000023f       0x33 ./MotorControl_Drivers/firmware/drivers/mss_usb/mss_usb_device_printer.o
 .ARM.attributes
                0x00000272       0x33 ./MotorControl_Drivers/firmware/drivers/mss_usb/mss_usb_device_vendor.o
 .ARM.attributes
                0x000002a5       0x33 ./MotorControl_Drivers/firmware/drivers/mss_usb/mss_usb_host.o
 .ARM.attributes
                0x000002d8       0x33 ./MotorControl_Drivers/firmware/drivers/mss_usb/mss_usb_host_cif.o
 .ARM.attributes
                0x0000030b       0x33 ./MotorControl_Drivers/firmware/drivers/mss_usb/mss_usb_host_msc.o
 .ARM.attributes
                0x0000033e       0x33 ./MotorControl_Drivers/firmware/drivers/mss_sys_services/mss_comblk.o
 .ARM.attributes
                0x00000371       0x33 ./MotorControl_Drivers/firmware/drivers/mss_sys_services/mss_sys_services.o
 .ARM.attributes
                0x000003a4       0x33 ./MotorControl_Drivers/firmware/drivers/mss_nvm/mss_nvm.o
 .ARM.attributes
                0x000003d7       0x33 ./MotorControl_Drivers/firmware/drivers/mss_hpdma/mss_hpdma.o
 .ARM.attributes
                0x0000040a       0x33 ./MotorControl_Drivers/firmware/drivers/mss_gpio/mss_gpio.o
 .ARM.attributes
                0x0000043d       0x33 ./MotorControl_Drivers/firmware/CMSIS/startup_gcc/newlib_stubs.o
 .ARM.attributes
                0x00000470       0x21 ./MotorControl_Drivers/firmware/CMSIS/startup_gcc/startup_m2sxxx.o
 .ARM.attributes
                0x00000491       0x33 ./MotorControl_Drivers/firmware/CMSIS/system_m2sxxx.o
 .ARM.attributes
                0x000004c4       0x33 ./MotorControl_App/MCCalc.o
 .ARM.attributes
                0x000004f7       0x33 ./MotorControl_App/MCFPGAIF.o
 .ARM.attributes
                0x0000052a       0x33 ./MotorControl_App/USBMsgHandler.o
 .ARM.attributes
                0x0000055d       0x33 ./MotorControl_App/main.o
 .ARM.attributes
                0x00000590       0x33 ./MotorControl_App/usb_user_descriptors.o
 .ARM.attributes
                0x000005c3       0x2d f:/microsemi/softconsole_v4.0/arm-none-eabi-gcc/bin/../lib/gcc/arm-none-eabi/4.9.3/../../../../arm-none-eabi/lib/armv7-m\libg_nano.a(lib_a-errno.o)
 .ARM.attributes
                0x000005f0       0x2d f:/microsemi/softconsole_v4.0/arm-none-eabi-gcc/bin/../lib/gcc/arm-none-eabi/4.9.3/../../../../arm-none-eabi/lib/armv7-m\libg_nano.a(lib_a-exit.o)
 .ARM.attributes
                0x0000061d       0x2d f:/microsemi/softconsole_v4.0/arm-none-eabi-gcc/bin/../lib/gcc/arm-none-eabi/4.9.3/../../../../arm-none-eabi/lib/armv7-m\libg_nano.a(lib_a-impure.o)
 .ARM.attributes
                0x0000064a       0x2d f:/microsemi/softconsole_v4.0/arm-none-eabi-gcc/bin/../lib/gcc/arm-none-eabi/4.9.3/../../../../arm-none-eabi/lib/armv7-m\libg_nano.a(lib_a-init.o)
 .ARM.attributes
                0x00000677       0x2d f:/microsemi/softconsole_v4.0/arm-none-eabi-gcc/bin/../lib/gcc/arm-none-eabi/4.9.3/../../../../arm-none-eabi/lib/armv7-m\libg_nano.a(lib_a-memcpy.o)
 .ARM.attributes
                0x000006a4       0x2d f:/microsemi/softconsole_v4.0/arm-none-eabi-gcc/bin/../lib/gcc/arm-none-eabi/4.9.3/../../../../arm-none-eabi/lib/armv7-m\libg_nano.a(lib_a-memset.o)
 .ARM.attributes
                0x000006d1       0x2d f:/microsemi/softconsole_v4.0/arm-none-eabi-gcc/bin/../lib/gcc/arm-none-eabi/4.9.3/armv7-m/crtend.o
 .ARM.attributes
                0x000006fe       0x1d f:/microsemi/softconsole_v4.0/arm-none-eabi-gcc/bin/../lib/gcc/arm-none-eabi/4.9.3/armv7-m/crtn.o

/DISCARD/
 *(.note.GNU-stack)
OUTPUT(MotorControl_5_1.elf elf32-littlearm)

.debug_ranges   0x00000000      0xe08
 .debug_ranges  0x00000000       0x38 ./MotorControl_Drivers/firmware/hal/CortexM3/cortex_nvic.o
 .debug_ranges  0x00000038      0x290 ./MotorControl_Drivers/firmware/drivers/mss_usb/mss_usb_common_cif.o
 .debug_ranges  0x000002c8      0x1f0 ./MotorControl_Drivers/firmware/drivers/mss_usb/mss_usb_device.o
 .debug_ranges  0x000004b8       0x68 ./MotorControl_Drivers/firmware/drivers/mss_usb/mss_usb_device_cdc.o
 .debug_ranges  0x00000520       0xf8 ./MotorControl_Drivers/firmware/drivers/mss_usb/mss_usb_device_cif.o
 .debug_ranges  0x00000618       0x70 ./MotorControl_Drivers/firmware/drivers/mss_usb/mss_usb_device_hid.o
 .debug_ranges  0x00000688       0xa8 ./MotorControl_Drivers/firmware/drivers/mss_usb/mss_usb_device_msd.o
 .debug_ranges  0x00000730       0x70 ./MotorControl_Drivers/firmware/drivers/mss_usb/mss_usb_device_printer.o
 .debug_ranges  0x000007a0       0x50 ./MotorControl_Drivers/firmware/drivers/mss_usb/mss_usb_device_vendor.o
 .debug_ranges  0x000007f0       0xd8 ./MotorControl_Drivers/firmware/drivers/mss_sys_services/mss_comblk.o
 .debug_ranges  0x000008c8      0x198 ./MotorControl_Drivers/firmware/drivers/mss_sys_services/mss_sys_services.o
 .debug_ranges  0x00000a60       0xb0 ./MotorControl_Drivers/firmware/drivers/mss_nvm/mss_nvm.o
 .debug_ranges  0x00000b10       0x80 ./MotorControl_Drivers/firmware/drivers/mss_hpdma/mss_hpdma.o
 .debug_ranges  0x00000b90       0x78 ./MotorControl_Drivers/firmware/drivers/mss_gpio/mss_gpio.o
 .debug_ranges  0x00000c08       0x98 ./MotorControl_Drivers/firmware/CMSIS/startup_gcc/newlib_stubs.o
 .debug_ranges  0x00000ca0       0x68 ./MotorControl_Drivers/firmware/CMSIS/system_m2sxxx.o
 .debug_ranges  0x00000d08       0x28 ./MotorControl_App/MCCalc.o
 .debug_ranges  0x00000d30       0x68 ./MotorControl_App/MCFPGAIF.o
 .debug_ranges  0x00000d98       0x38 ./MotorControl_App/USBMsgHandler.o
 .debug_ranges  0x00000dd0       0x10 ./MotorControl_App/main.o
 .debug_ranges  0x00000de0       0x28 ./MotorControl_App/usb_user_descriptors.o

.comment        0x00000000       0x70
 .comment       0x00000000       0x70 ./MotorControl_Drivers/firmware/hal/CortexM3/cortex_nvic.o
                                 0x71 (size before relaxing)
 .comment       0x00000000       0x71 ./MotorControl_Drivers/firmware/drivers_config/sys_config/sys_config.o
 .comment       0x00000000       0x71 ./MotorControl_Drivers/firmware/drivers/mss_usb/mss_usb_common_cif.o
 .comment       0x00000000       0x71 ./MotorControl_Drivers/firmware/drivers/mss_usb/mss_usb_device.o
 .comment       0x00000000       0x71 ./MotorControl_Drivers/firmware/drivers/mss_usb/mss_usb_device_cdc.o
 .comment       0x00000000       0x71 ./MotorControl_Drivers/firmware/drivers/mss_usb/mss_usb_device_cif.o
 .comment       0x00000000       0x71 ./MotorControl_Drivers/firmware/drivers/mss_usb/mss_usb_device_hid.o
 .comment       0x00000000       0x71 ./MotorControl_Drivers/firmware/drivers/mss_usb/mss_usb_device_msd.o
 .comment       0x00000000       0x71 ./MotorControl_Drivers/firmware/drivers/mss_usb/mss_usb_device_printer.o
 .comment       0x00000000       0x71 ./MotorControl_Drivers/firmware/drivers/mss_usb/mss_usb_device_vendor.o
 .comment       0x00000000       0x71 ./MotorControl_Drivers/firmware/drivers/mss_usb/mss_usb_host.o
 .comment       0x00000000       0x71 ./MotorControl_Drivers/firmware/drivers/mss_usb/mss_usb_host_cif.o
 .comment       0x00000000       0x71 ./MotorControl_Drivers/firmware/drivers/mss_usb/mss_usb_host_msc.o
 .comment       0x00000000       0x71 ./MotorControl_Drivers/firmware/drivers/mss_sys_services/mss_comblk.o
 .comment       0x00000000       0x71 ./MotorControl_Drivers/firmware/drivers/mss_sys_services/mss_sys_services.o
 .comment       0x00000000       0x71 ./MotorControl_Drivers/firmware/drivers/mss_nvm/mss_nvm.o
 .comment       0x00000000       0x71 ./MotorControl_Drivers/firmware/drivers/mss_hpdma/mss_hpdma.o
 .comment       0x00000000       0x71 ./MotorControl_Drivers/firmware/drivers/mss_gpio/mss_gpio.o
 .comment       0x00000000       0x71 ./MotorControl_Drivers/firmware/CMSIS/startup_gcc/newlib_stubs.o
 .comment       0x00000000       0x71 ./MotorControl_Drivers/firmware/CMSIS/system_m2sxxx.o
 .comment       0x00000000       0x71 ./MotorControl_App/MCCalc.o
 .comment       0x00000000       0x71 ./MotorControl_App/MCFPGAIF.o
 .comment       0x00000000       0x71 ./MotorControl_App/USBMsgHandler.o
 .comment       0x00000000       0x71 ./MotorControl_App/main.o
 .comment       0x00000000       0x71 ./MotorControl_App/usb_user_descriptors.o
